BL51 BANKED LINKER/LOCATER V4.02                                                        05/28/2008  17:48:13  PAGE 1


BL51 BANKED LINKER/LOCATER V4.02, INVOKED BY:
E:\BRNO\ZALOHA\DISK_C\ATMEL\C51\KEIL6\C51\BIN\BL51.EXE main.obj, main_routines.obj, LCD_functions.obj, LCD_routines.obj,
>>  text_graphics_functions.obj, text_graphics_routines.obj, fonts.obj, buttons.obj, MODBUS.obj, MODBUS_routines.obj, E3
>> D_demo.obj, screens.obj, user_actions.obj TO LCD_terminal CODE (0X0000-0XFFFE) XDATA (0X0000-0X7FFF)


MEMORY MODEL: SMALL


INPUT MODULES INCLUDED:
  main.obj (MAIN)
  main_routines.obj (MAIN_ROUTINES)
  LCD_functions.obj (LCD_FUNCTIONS)
  LCD_routines.obj (LCD_ROUTINES)
  text_graphics_functions.obj (TEXT_GRAPHICS_FUNCTIONS)
  text_graphics_routines.obj (TXT_GRAPH)
  fonts.obj (FONTS)
  buttons.obj (BUTTONS)
  MODBUS.obj (MODBUS)
  MODBUS_routines.obj (MODBUS_ROUTINES)
  E3D_demo.obj (E3D_DEMO)
  screens.obj (SCREENS)
  user_actions.obj (USER_ACTIONS)
  E:\BRNO\ZALOHA\DISK_C\ATMEL\C51\KEIL6\C51\LIB\C51S.LIB (?C_STARTUP)
  E:\BRNO\ZALOHA\DISK_C\ATMEL\C51\KEIL6\C51\LIB\C51S.LIB (?C?COPY)
  E:\BRNO\ZALOHA\DISK_C\ATMEL\C51\KEIL6\C51\LIB\C51S.LIB (?C?CLDPTR)
  E:\BRNO\ZALOHA\DISK_C\ATMEL\C51\KEIL6\C51\LIB\C51S.LIB (?C?CILDPTR)
  E:\BRNO\ZALOHA\DISK_C\ATMEL\C51\KEIL6\C51\LIB\C51S.LIB (?C?CSTPTR)
  E:\BRNO\ZALOHA\DISK_C\ATMEL\C51\KEIL6\C51\LIB\C51S.LIB (?C?IMUL)
  E:\BRNO\ZALOHA\DISK_C\ATMEL\C51\KEIL6\C51\LIB\C51S.LIB (?C?SIDIV)
  E:\BRNO\ZALOHA\DISK_C\ATMEL\C51\KEIL6\C51\LIB\C51S.LIB (?C?ILDIX)
  E:\BRNO\ZALOHA\DISK_C\ATMEL\C51\KEIL6\C51\LIB\C51S.LIB (?C?ILDPTR)
  E:\BRNO\ZALOHA\DISK_C\ATMEL\C51\KEIL6\C51\LIB\C51S.LIB (?C?IILDPTR)
  E:\BRNO\ZALOHA\DISK_C\ATMEL\C51\KEIL6\C51\LIB\C51S.LIB (?C?ISTPTR)
  E:\BRNO\ZALOHA\DISK_C\ATMEL\C51\KEIL6\C51\LIB\C51S.LIB (?C?ISTOPTR)
  E:\BRNO\ZALOHA\DISK_C\ATMEL\C51\KEIL6\C51\LIB\C51S.LIB (?C?LMUL)
  E:\BRNO\ZALOHA\DISK_C\ATMEL\C51\KEIL6\C51\LIB\C51S.LIB (?C?SLDIV)
  E:\BRNO\ZALOHA\DISK_C\ATMEL\C51\KEIL6\C51\LIB\C51S.LIB (?C?SLSHR)
  E:\BRNO\ZALOHA\DISK_C\ATMEL\C51\KEIL6\C51\LIB\C51S.LIB (?C?OFFXADD)
  E:\BRNO\ZALOHA\DISK_C\ATMEL\C51\KEIL6\C51\LIB\C51S.LIB (?C?PSTOPTR)
  E:\BRNO\ZALOHA\DISK_C\ATMEL\C51\KEIL6\C51\LIB\C51S.LIB (?C?ICALL)
  E:\BRNO\ZALOHA\DISK_C\ATMEL\C51\KEIL6\C51\LIB\C51S.LIB (PRINTF)
  E:\BRNO\ZALOHA\DISK_C\ATMEL\C51\KEIL6\C51\LIB\C51S.LIB (RAND)
  E:\BRNO\ZALOHA\DISK_C\ATMEL\C51\KEIL6\C51\LIB\C51S.LIB (?C?STRCPY)
  E:\BRNO\ZALOHA\DISK_C\ATMEL\C51\KEIL6\C51\LIB\C51S.LIB (?C?MEMSET)
  E:\BRNO\ZALOHA\DISK_C\ATMEL\C51\KEIL6\C51\LIB\C51S.LIB (?C_INIT)
  E:\BRNO\ZALOHA\DISK_C\ATMEL\C51\KEIL6\C51\LIB\C51S.LIB (?C?CLDOPTR)
  E:\BRNO\ZALOHA\DISK_C\ATMEL\C51\KEIL6\C51\LIB\C51S.LIB (?C?UIDIV)
  E:\BRNO\ZALOHA\DISK_C\ATMEL\C51\KEIL6\C51\LIB\C51S.LIB (?C?IILDX)
  E:\BRNO\ZALOHA\DISK_C\ATMEL\C51\KEIL6\C51\LIB\C51S.LIB (?C?ULDIV)
  E:\BRNO\ZALOHA\DISK_C\ATMEL\C51\KEIL6\C51\LIB\C51S.LIB (?C?PLDIIDATA)
  E:\BRNO\ZALOHA\DISK_C\ATMEL\C51\KEIL6\C51\LIB\C51S.LIB (?C?PSTIDATA)
  E:\BRNO\ZALOHA\DISK_C\ATMEL\C51\KEIL6\C51\LIB\C51S.LIB (?C?PSTXDATA)
  E:\BRNO\ZALOHA\DISK_C\ATMEL\C51\KEIL6\C51\LIB\C51S.LIB (?C?PSTPDATA)
  E:\BRNO\ZALOHA\DISK_C\ATMEL\C51\KEIL6\C51\LIB\C51S.LIB (?C?CCASE)
  E:\BRNO\ZALOHA\DISK_C\ATMEL\C51\KEIL6\C51\LIB\C51S.LIB (PUTCHAR)


BL51 BANKED LINKER/LOCATER V4.02                                                      05/28/2008  17:48:13  PAGE 2


LINK MAP OF MODULE:  LCD_terminal (MAIN)


            TYPE    BASE      LENGTH    RELOCATION   SEGMENT NAME
            -----------------------------------------------------

            * * * * * * *   D A T A   M E M O R Y   * * * * * * *
            REG     0000H     0008H     ABSOLUTE     "REG BANK 0"
            DATA    0008H     0006H     UNIT         ?DT?_DRAWICON?TXT_GRAPH
            DATA    000EH     0002H     UNIT         ?DT?MAIN
            REG     0010H     0008H     ABSOLUTE     "REG BANK 2"
            REG     0018H     0008H     ABSOLUTE     "REG BANK 3"
            BIT     0020H.0   0001H.1   UNIT         _BIT_GROUP_
                    0021H.1   0000H.7                *** GAP ***
            DATA    0022H     0014H     UNIT         _DATA_GROUP_
            DATA    0036H     0004H     UNIT         ?DT?_DRAWLINE?TXT_GRAPH
            DATA    003AH     0004H     UNIT         ?DT?BUTTONS
            DATA    003EH     0004H     UNIT         ?DT?RAND?RAND
            DATA    0042H     0001H     UNIT         ?DT?MODBUS
            IDATA   0043H     0001H     UNIT         ?STACK

            * * * * * * *  X D A T A   M E M O R Y  * * * * * * *
            XDATA   0000H     1300H     UNIT         ?XD?MAIN
            XDATA   1300H     0206H     UNIT         ?XD?MODBUS
            XDATA   1506H     01D4H     UNIT         ?XD?BUTTONS
            XDATA   16DAH     003EH     UNIT         ?XD?E3D_DEMO
            XDATA   1718H     0028H     UNIT         _XDATA_GROUP_
            XDATA   1740H     0001H     UNIT         ?XD?USER_ACTIONS

            * * * * * * *   C O D E   M E M O R Y   * * * * * * *
            CODE    0000H     0003H     ABSOLUTE     
            CODE    0003H     0008H     UNIT         ?CO?TEXT_GRAPHICS_FUNCTIONS
            CODE    000BH     0003H     ABSOLUTE     
            CODE    000EH     0009H     UNIT         ?CO?BUTTONS
            CODE    0017H     0003H     UNIT         ?PR?ACTBACKLEDOFF?USER_ACTIONS
                    001AH     0001H                  *** GAP ***
            CODE    001BH     0003H     ABSOLUTE     
            CODE    001EH     0003H     UNIT         ?PR?ACTBACKLEDON?USER_ACTIONS
                    0021H     0002H                  *** GAP ***
            CODE    0023H     0003H     ABSOLUTE     
            CODE    0026H     2841H     UNIT         CODESEG
            CODE    2867H     06FDH     UNIT         ?CO?SCREENS
            CODE    2F64H     05EAH     UNIT         ?C?LIB_CODE
            CODE    354EH     03CCH     UNIT         ?CO?E3D_DEMO
            CODE    391AH     03C2H     UNIT         ?PR?MODBUS?MODBUS
            CODE    3CDCH     035CH     UNIT         ?PR?PRINTF?PRINTF
            CODE    4038H     025FH     UNIT         ?PR?_E3D_RANDOMMOVE?E3D_DEMO
            CODE    4297H     024DH     UNIT         ?PR?_E3D_MAKE_MOVE_ROTATE_TRANSFORM?E3D_DEMO
            CODE    44E4H     0224H     UNIT         ?PR?_CRC16?MODBUS_ROUTINES
            CODE    4708H     01D2H     UNIT         ?PR?GUI?BUTTONS
            CODE    48DAH     01B8H     UNIT         ?PR?_SCREEN3?SCREENS
            CODE    4A92H     018CH     UNIT         ?PR?E3D_DEMO
            CODE    4C1EH     011BH     UNIT         ?PR?_DRAWLINE?TXT_GRAPH
            CODE    4D39H     00FCH     UNIT         ?PR?_DRAWSTRXRAM?TXT_GRAPH
            CODE    4E35H     00FCH     UNIT         ?PR?MODBUS
            CODE    4F31H     00DCH     UNIT         ?PR?_DRAWSTRBCK?TXT_GRAPH
            CODE    500DH     00DBH     UNIT         ?PR?_SCREEN2?SCREENS
BL51 BANKED LINKER/LOCATER V4.02                                                      05/28/2008  17:48:13  PAGE 3


            CODE    50E8H     00AAH     UNIT         ?PR?_SCREEN1?SCREENS
            CODE    5192H     0095H     UNIT         ?PR?_ADDACTION?BUTTONS
            CODE    5227H     0092H     UNIT         ?PR?_DRAWFRAME?TEXT_GRAPHICS_FUNCTIONS
            CODE    52B9H     008DH     UNIT         ?PR?_E3D_ROTATE?E3D_DEMO
            CODE    5346H     008CH     UNIT         ?C_C51STARTUP
            CODE    53D2H     007BH     UNIT         ?PR?_DRAWICON?TXT_GRAPH
            CODE    544DH     0074H     UNIT         ?PR?INT_UART?MODBUS
            CODE    54C1H     0073H     UNIT         ?PR?_E3D_DRAWOBJECT?E3D_DEMO
            CODE    5534H     0062H     UNIT         ?PR?INTTIMER0?BUTTONS
            CODE    5596H     0061H     UNIT         ?PR?_DRAWSTRING?TEXT_GRAPHICS_FUNCTIONS
            CODE    55F7H     0060H     UNIT         ?PR?_E3D_DEMO?E3D_DEMO
            CODE    5657H     005CH     UNIT         ?CO?MODBUS
            CODE    56B3H     0052H     UNIT         ?PR?BUTTONS
            CODE    5705H     0044H     UNIT         ?PR?ACTLEDBLINK?USER_ACTIONS
            CODE    5749H     0044H     UNIT         ?C?LDIV
            CODE    578DH     0041H     UNIT         ?PR?RAND?RAND
            CODE    57CEH     0040H     UNIT         ?PR?MAIN?MAIN
            CODE    580EH     003BH     UNIT         ?C_INITSEG
            CODE    5849H     003BH     UNIT         ?PR?MODBUSINIT?MODBUS
            CODE    5884H     0030H     UNIT         ?PR?LCDINIT?LCD_FUNCTIONS
            CODE    58B4H     0028H     UNIT         ?PR?SCREENS
            CODE    58DCH     0027H     UNIT         ?PR?PUTCHAR?PUTCHAR
            CODE    5903H     0015H     UNIT         ?PR?BUTTONSINIT?BUTTONS
            CODE    5918H     000FH     UNIT         ?PR?MAIN
            CODE    5927H     000FH     UNIT         ?PR?CLEARACTIONS?BUTTONS
            CODE    5936H     000FH     UNIT         ?PR?INT_TIMER1?MODBUS



OVERLAY MAP OF MODULE:   LCD_terminal (MAIN)


SEGMENT                                                 BIT_GROUP          DATA_GROUP          XDATA_GROUP
  +--> CALLED SEGMENT                                START    LENGTH     START    LENGTH     START    LENGTH
------------------------------------------------------------------------------------------------------------
?PR?INTTIMER0?BUTTONS                                -----    -----      -----    -----      -----    -----
  +--> ?PR?BUTTONS
  +--> ?PR?_E3D_DEMO?E3D_DEMO

?PR?_E3D_DEMO?E3D_DEMO                               -----    -----      -----    -----      -----    -----
  +--> ?PR?CLEARACTIONS?BUTTONS
  +--> ?PR?_ADDACTION?BUTTONS
  +--> ?PR?_E3D_MAKE_MOVE_ROTATE_TRANSFORM?E3D_DEMO
  +--> ?PR?_E3D_DRAWOBJECT?E3D_DEMO
  +--> ?PR?_E3D_ROTATE?E3D_DEMO
  +--> ?PR?_E3D_RANDOMMOVE?E3D_DEMO

?PR?_ADDACTION?BUTTONS                               -----    -----      -----    -----      172CH    000EH
  +--> ?PR?BUTTONS
  +--> ?CO?BUTTONS

?PR?_E3D_MAKE_MOVE_ROTATE_TRANSFORM?E3D_DEMO         -----    -----      -----    -----      172CH    0014H
  +--> ?PR?E3D_DEMO
  +--> ?CO?E3D_DEMO

?PR?E3D_DEMO                                         -----    -----      -----    -----      -----    -----
  +--> ?CO?E3D_DEMO
BL51 BANKED LINKER/LOCATER V4.02                                                      05/28/2008  17:48:13  PAGE 4



?PR?_E3D_DRAWOBJECT?E3D_DEMO                         -----    -----      -----    -----      172CH    0004H
  +--> ?PR?E3D_DEMO
  +--> ?PR?_DRAWLINE?TXT_GRAPH

?PR?_E3D_ROTATE?E3D_DEMO                             -----    -----      -----    -----      172CH    0003H
  +--> ?PR?E3D_DEMO

?PR?_E3D_RANDOMMOVE?E3D_DEMO                         -----    -----      -----    -----      172CH    000FH
  +--> ?PR?E3D_DEMO
  +--> ?PR?RAND?RAND

*** NEW ROOT ***************************************************

?PR?INT_TIMER1?MODBUS                                -----    -----      -----    -----      -----    -----
  +--> ?PR?MODBUS

*** NEW ROOT ***************************************************

?PR?INT_UART?MODBUS                                  -----    -----      -----    -----      -----    -----
  +--> ?PR?MODBUS

*** NEW ROOT ***************************************************

?C_C51STARTUP                                        -----    -----      -----    -----      -----    -----
  +--> ?PR?MAIN?MAIN
  +--> ?C_INITSEG

?PR?MAIN?MAIN                                        -----    -----      -----    -----      -----    -----
  +--> ?PR?CLEARACTIONS?BUTTONS
  +--> ?PR?BUTTONSINIT?BUTTONS
  +--> ?PR?LCDINIT?LCD_FUNCTIONS
  +--> ?PR?MODBUSINIT?MODBUS
  +--> ?PR?MAIN
  +--> ?PR?_SCREEN1?SCREENS
  +--> ?PR?_SCREEN2?SCREENS
  +--> ?PR?RAND?RAND
  +--> ?PR?GUI?BUTTONS
  +--> ?PR?MODBUS?MODBUS

?PR?MODBUSINIT?MODBUS                                -----    -----      -----    -----      -----    -----
  +--> ?PR?MODBUS

?PR?_SCREEN1?SCREENS                                 -----    -----      -----    -----      -----    -----
  +--> ?PR?SCREENS
  +--> ?PR?CLEARACTIONS?BUTTONS
  +--> ?PR?_ADDACTION?BUTTONS
  +--> ?CO?SCREENS
  +--> ?PR?_DRAWSTRING?TEXT_GRAPHICS_FUNCTIONS
  +--> ?PR?_DRAWICON?TXT_GRAPH
  +--> ?PR?_DRAWFRAME?TEXT_GRAPHICS_FUNCTIONS

?PR?_DRAWSTRING?TEXT_GRAPHICS_FUNCTIONS              -----    -----      0022H    0007H      -----    -----
  +--> ?CO?TEXT_GRAPHICS_FUNCTIONS
  +--> ?PR?_DRAWSTRXRAM?TXT_GRAPH

?PR?_DRAWSTRXRAM?TXT_GRAPH                           -----    -----      -----    -----      -----    -----
BL51 BANKED LINKER/LOCATER V4.02                                                      05/28/2008  17:48:13  PAGE 5


  +--> ?PR?_DRAWSTRBCK?TXT_GRAPH

?PR?_DRAWFRAME?TEXT_GRAPHICS_FUNCTIONS               -----    -----      0022H    0005H      -----    -----
  +--> ?PR?_DRAWLINE?TXT_GRAPH

?PR?_SCREEN2?SCREENS                                 -----    -----      -----    -----      -----    -----
  +--> ?PR?SCREENS
  +--> ?PR?CLEARACTIONS?BUTTONS
  +--> ?PR?_SCREEN1?SCREENS
  +--> ?PR?_ADDACTION?BUTTONS
  +--> ?PR?_SCREEN3?SCREENS
  +--> ?PR?_E3D_DEMO?E3D_DEMO
  +--> ?CO?SCREENS
  +--> ?PR?_DRAWICON?TXT_GRAPH
  +--> ?PR?_DRAWSTRING?TEXT_GRAPHICS_FUNCTIONS

?PR?_SCREEN3?SCREENS                                 -----    -----      -----    -----      -----    -----
  +--> ?PR?SCREENS
  +--> ?PR?CLEARACTIONS?BUTTONS
  +--> ?PR?_ADDACTION?BUTTONS
  +--> ?PR?ACTLEDBLINK?USER_ACTIONS
  +--> ?PR?ACTBACKLEDOFF?USER_ACTIONS
  +--> ?PR?ACTBACKLEDON?USER_ACTIONS
  +--> ?PR?_DRAWFRAME?TEXT_GRAPHICS_FUNCTIONS
  +--> ?CO?SCREENS
  +--> ?PR?_DRAWSTRING?TEXT_GRAPHICS_FUNCTIONS
  +--> ?PR?_DRAWLINE?TXT_GRAPH
  +--> ?PR?PRINTF?PRINTF

?PR?ACTLEDBLINK?USER_ACTIONS                         -----    -----      -----    -----      172CH    0002H

?PR?PRINTF?PRINTF                                    0020H.0  0001H.1    0022H    0014H      -----    -----
  +--> ?PR?PUTCHAR?PUTCHAR

?PR?GUI?BUTTONS                                      -----    -----      0022H    0001H      172CH    000AH
  +--> ?PR?BUTTONS

?PR?MODBUS?MODBUS                                    -----    -----      -----    -----      172CH    0008H
  +--> ?PR?_CRC16?MODBUS_ROUTINES
  +--> ?PR?MODBUS
  +--> ?CO?MODBUS

?C_INITSEG                                           -----    -----      -----    -----      -----    -----
  +--> ?CO?E3D_DEMO



SYMBOL TABLE OF MODULE:  LCD_terminal (MAIN)

  VALUE           TYPE          NAME
  ----------------------------------

  -------         MODULE        MAIN
  C:0000H         SYMBOL        _ICE_DUMMY_
  B:00D8H.2       PUBLIC        CCF2
  B:00D8H.3       PUBLIC        CCF3
  B:00D8H.4       PUBLIC        CCF4
BL51 BANKED LINKER/LOCATER V4.02                                                      05/28/2008  17:48:13  PAGE 6


  B:00D0H.6       PUBLIC        AC
  B:00B0H.4       PUBLIC        T0
  B:00B0H.5       PUBLIC        T1
  B:00A8H.7       PUBLIC        EA
  B:00A8H.6       PUBLIC        EC
  B:00D8H.7       PUBLIC        CF
  B:0098H.7       PUBLIC        FE
  B:00E8H.1       PUBLIC        EADC
  B:0080H.0       PUBLIC        P0_0
  B:0090H.0       PUBLIC        P1_0
  B:0080H.1       PUBLIC        P0_1
  B:00A0H.0       PUBLIC        P2_0
  B:0090H.1       PUBLIC        P1_1
  B:0080H.2       PUBLIC        P0_2
  B:00B0H.0       PUBLIC        P3_0
  B:00A0H.1       PUBLIC        P2_1
  B:0090H.2       PUBLIC        P1_2
  B:0080H.3       PUBLIC        P0_3
  B:00C0H.0       PUBLIC        P4_0
  B:00B0H.1       PUBLIC        P3_1
  B:00A0H.2       PUBLIC        P2_2
  B:0090H.3       PUBLIC        P1_3
  B:0080H.4       PUBLIC        P0_4
  B:00D8H.6       PUBLIC        CR
  B:00C0H.1       PUBLIC        P4_1
  B:00B0H.2       PUBLIC        P3_2
  B:00A0H.3       PUBLIC        P2_3
  B:0090H.4       PUBLIC        P1_4
  B:0080H.5       PUBLIC        P0_5
  B:00C8H.6       PUBLIC        EXF2
  B:00B0H.7       PUBLIC        RD
  B:00B0H.3       PUBLIC        P3_3
  B:00A0H.4       PUBLIC        P2_4
  B:0090H.5       PUBLIC        P1_5
  B:0080H.6       PUBLIC        P0_6
  B:00B0H.4       PUBLIC        P3_4
  B:00A0H.5       PUBLIC        P2_5
  B:0090H.6       PUBLIC        P1_6
  B:0080H.7       PUBLIC        P0_7
  B:00E8H.0       PUBLIC        ECAN
  B:00A8H.4       PUBLIC        ES
  B:00B0H.5       PUBLIC        P3_5
  B:00A0H.6       PUBLIC        P2_6
  B:0090H.7       PUBLIC        P1_7
  B:00D0H.1       PUBLIC        UD
  B:00B0H.6       PUBLIC        P3_6
  B:00A0H.7       PUBLIC        P2_7
  B:00B0H.7       PUBLIC        P3_7
  B:0098H.0       PUBLIC        RI
  B:00D0H.7       PUBLIC        CY
  B:00B0H.2       PUBLIC        INT0
  B:0098H.1       PUBLIC        TI
  B:00B0H.3       PUBLIC        INT1
  B:00D0H.2       PUBLIC        OV
  C:57CEH         PUBLIC        main
  B:00C8H.1       PUBLIC        C_T2
  B:00B0H.6       PUBLIC        WR
BL51 BANKED LINKER/LOCATER V4.02                                                      05/28/2008  17:48:13  PAGE 7


  B:00C8H.5       PUBLIC        RCLK
  X:0000H         PUBLIC        strtmp
  B:00C8H.4       PUBLIC        TCLK
  B:00E8H.2       PUBLIC        ETIM
  B:00E8H.3       PUBLIC        ESPI
  B:0088H.1       PUBLIC        IE0
  B:0088H.3       PUBLIC        IE1
  D:008EH         PUBLIC        AUXR
  B:00C8H.0       PUBLIC        CP_RL2
  B:00A8H.1       PUBLIC        ET0
  B:00A8H.3       PUBLIC        ET1
  B:0088H.5       PUBLIC        TF0
  B:00A8H.5       PUBLIC        ET2
  B:0088H.7       PUBLIC        TF1
  D:000EH         PUBLIC        xpos
  B:0098H.2       PUBLIC        RB8
  B:00C8H.7       PUBLIC        TF2
  D:000FH         PUBLIC        ypos
  B:00A8H.0       PUBLIC        EX0
  B:0088H.0       PUBLIC        IT0
  B:00A8H.2       PUBLIC        EX1
  B:0098H.3       PUBLIC        TB8
  B:0088H.2       PUBLIC        IT1
  B:00D0H.0       PUBLIC        P
  B:0098H.7       PUBLIC        SM0
  B:0098H.6       PUBLIC        SM1
  B:0098H.5       PUBLIC        SM2
  B:00D0H.3       PUBLIC        RS0
  B:0088H.4       PUBLIC        TR0
  B:00D0H.4       PUBLIC        RS1
  B:0088H.6       PUBLIC        TR1
  B:00C8H.2       PUBLIC        TR2
  B:00C8H.3       PUBLIC        EXEN2
  B:0098H.4       PUBLIC        REN
  X:0400H         PUBLIC        img0
  B:00B0H.0       PUBLIC        RXD
  D:008FH         PUBLIC        CKCON
  B:00B0H.1       PUBLIC        TXD
  B:00D0H.5       PUBLIC        F0
  B:00D8H.0       PUBLIC        CCF0
  B:00D8H.1       PUBLIC        CCF1
  -------         PROC          COM0004
  -------         ENDPROC       COM0004
  -------         PROC          MAIN
  C:57CEH         LINE#         27
  C:57CEH         LINE#         28
  C:57CEH         LINE#         31
  C:57D1H         LINE#         32
  C:57D4H         LINE#         35
  C:57D6H         LINE#         38
  C:57D9H         LINE#         41
  C:57DCH         LINE#         44
  C:57DFH         LINE#         47
  C:57E2H         LINE#         50
  C:57E4H         LINE#         53
  C:57E7H         LINE#         54
  C:57ECH         LINE#         55
BL51 BANKED LINKER/LOCATER V4.02                                                      05/28/2008  17:48:13  PAGE 8


  C:57EFH         LINE#         56
  C:57F4H         LINE#         59
  C:57F7H         LINE#         60
  C:57FCH         LINE#         61
  C:57FFH         LINE#         63
  C:5806H         LINE#         66
  C:5806H         LINE#         67
  C:5806H         LINE#         69
  C:5809H         LINE#         71
  C:580CH         LINE#         72
  -------         ENDPROC       MAIN
  -------         ENDMOD        MAIN

  -------         MODULE        MAIN_ROUTINES
  C:0026H         SEGMENT       CODESEG
  C:0034H         PUBLIC        _CPOW2
  C:0026H         PUBLIC        _DELAY10MS
  D:00E0H         SYMBOL        ACC
  D:00F0H         SYMBOL        B
  C:003DH         SYMBOL        CPOW2S1
  C:0041H         SYMBOL        CPOW2S2
  C:0045H         SYMBOL        CPOW2S3
  C:0028H         SYMBOL        DELAY10MSL1
  N:0000H         SYMBOL        MAIN_ROUTINES
  C:0026H         LINE#         16
  C:0028H         LINE#         17
  C:002BH         LINE#         18
  C:002EH         LINE#         19
  C:0031H         LINE#         20
  C:0033H         LINE#         21
  C:0034H         LINE#         34
  C:0036H         LINE#         35
  C:0038H         LINE#         36
  C:003BH         LINE#         37
  C:003DH         LINE#         38
  C:0040H         LINE#         39
  C:0041H         LINE#         40
  C:0044H         LINE#         41
  C:0045H         LINE#         42
  C:0046H         LINE#         43
  -------         ENDMOD        MAIN_ROUTINES

  -------         MODULE        LCD_FUNCTIONS
  C:0000H         SYMBOL        _ICE_DUMMY_
  C:5884H         PUBLIC        LCDinit
  -------         PROC          LCDINIT
  C:5884H         LINE#         7
  C:5884H         LINE#         8
  C:5884H         LINE#         9
  C:5887H         LINE#         10
  C:588FH         LINE#         11
  C:5898H         LINE#         12
  C:58A1H         LINE#         13
  C:58AAH         LINE#         14
  C:58AFH         LINE#         15
  -------         ENDPROC       LCDINIT
  -------         ENDMOD        LCD_FUNCTIONS
BL51 BANKED LINKER/LOCATER V4.02                                                      05/28/2008  17:48:13  PAGE 9



  -------         MODULE        LCD_ROUTINES
  C:0026H         SEGMENT       CODESEG
  C:0093H         PUBLIC        LCDDRAWIMG
  C:007FH         PUBLIC        LCDRESET
  C:0074H         PUBLIC        LCDWAITSTAT
  C:0047H         PUBLIC        _LCDTXCMD
  C:004FH         PUBLIC        _LCDTXCMDP1
  C:005EH         PUBLIC        _LCDTXCMDP2
  D:00E0H         SYMBOL        ACC
  D:00A2H         SYMBOL        AUXR1
  D:00F0H         SYMBOL        B
  D:0083H         SYMBOL        DPH
  D:0082H         SYMBOL        DPL
  C:00AEH         SYMBOL        LCDDRAWIMGL1
  C:0085H         SYMBOL        LCDRESETL1
  C:0083H         SYMBOL        LCDRESETL2
  C:0077H         SYMBOL        LCDWAITSTATL1
  N:9000H         SYMBOL        LCD_ADDR_CMD
  N:8000H         SYMBOL        LCD_ADDR_DATA
  N:0500H         SYMBOL        LCD_RAM_BASE
  N:0000H         SYMBOL        LCD_ROUTINES
  B:00C0H.0       SYMBOL        LRST
  N:00C0H         SYMBOL        P4
  C:00BDH         SYMBOL        WRITEIMG1S1
  C:00ABH         SYMBOL        WRITEIMGIMG1
  C:00A9H         SYMBOL        WRITEIMGIMG2
  C:0047H         LINE#         22
  C:0049H         LINE#         23
  C:004CH         LINE#         24
  C:004DH         LINE#         25
  C:004EH         LINE#         26
  C:004FH         LINE#         33
  C:0051H         LINE#         34
  C:0054H         LINE#         35
  C:0055H         LINE#         36
  C:0056H         LINE#         37
  C:0058H         LINE#         38
  C:005BH         LINE#         39
  C:005CH         LINE#         40
  C:005DH         LINE#         41
  C:005EH         LINE#         48
  C:0060H         LINE#         49
  C:0063H         LINE#         50
  C:0064H         LINE#         51
  C:0065H         LINE#         52
  C:0067H         LINE#         53
  C:006AH         LINE#         54
  C:006BH         LINE#         55
  C:006CH         LINE#         56
  C:006EH         LINE#         57
  C:0071H         LINE#         58
  C:0072H         LINE#         59
  C:0073H         LINE#         60
  C:0074H         LINE#         67
  C:0077H         LINE#         68
  C:0078H         LINE#         69
BL51 BANKED LINKER/LOCATER V4.02                                                      05/28/2008  17:48:13  PAGE 10


  C:007BH         LINE#         70
  C:007EH         LINE#         71
  C:007FH         LINE#         81
  C:0081H         LINE#         82
  C:0083H         LINE#         83
  C:0085H         LINE#         84
  C:0088H         LINE#         85
  C:008BH         LINE#         86
  C:008EH         LINE#         87
  C:0090H         LINE#         88
  C:0092H         LINE#         89
  C:0093H         LINE#         101
  C:0095H         LINE#         102
  C:0097H         LINE#         103
  C:0099H         LINE#         104
  C:009BH         LINE#         105
  C:009DH         LINE#         106
  C:009FH         LINE#         108
  C:00A2H         LINE#         109
  C:00A4H         LINE#         110
  C:00A7H         LINE#         112
  C:00A9H         LINE#         113
  C:00ABH         LINE#         115
  C:00AEH         LINE#         116
  C:00AFH         LINE#         117
  C:00B2H         LINE#         119
  C:00B4H         LINE#         120
  C:00B6H         LINE#         121
  C:00B8H         LINE#         122
  C:00BBH         LINE#         123
  C:00BDH         LINE#         124
  C:00BEH         LINE#         125
  C:00C0H         LINE#         127
  C:00C3H         LINE#         128
  C:00C4H         LINE#         130
  C:00C6H         LINE#         131
  C:00C8H         LINE#         132
  C:00CAH         LINE#         134
  C:00CCH         LINE#         135
  C:00CEH         LINE#         136
  -------         ENDMOD        LCD_ROUTINES

  -------         MODULE        TEXT_GRAPHICS_FUNCTIONS
  C:0000H         SYMBOL        _ICE_DUMMY_
  C:5227H         PUBLIC        _DrawFrame
  C:5596H         PUBLIC        _DrawString
  -------         PROC          _DRAWSTRING
  D:0007H         SYMBOL        x
  D:0005H         SYMBOL        y
  D:0024H         SYMBOL        font
  D:0025H         SYMBOL        btn
  D:0026H         SYMBOL        str
  -------         DO            str
  C:0003H         SYMBOL        btnmap
  -------         ENDDO         btnmap
  C:5596H         LINE#         10
  C:5598H         LINE#         11
BL51 BANKED LINKER/LOCATER V4.02                                                      05/28/2008  17:48:13  PAGE 11


  C:5598H         LINE#         14
  C:55A1H         LINE#         15
  C:55AAH         LINE#         17
  C:55B2H         LINE#         18
  C:55C1H         LINE#         20
  -------         ENDPROC       _DRAWSTRING
  -------         PROC          _DRAWFRAME
  D:0022H         SYMBOL        Ax
  D:0023H         SYMBOL        Ay
  D:0024H         SYMBOL        Bx
  D:0025H         SYMBOL        By
  D:0026H         SYMBOL        style
  C:5227H         LINE#         26
  C:522DH         LINE#         27
  C:522DH         LINE#         28
  C:5249H         LINE#         29
  C:5249H         LINE#         30
  C:524EH         LINE#         31
  C:524EH         LINE#         32
  C:5255H         LINE#         33
  C:5265H         LINE#         34
  C:5265H         LINE#         36
  C:5265H         LINE#         37
  C:5265H         LINE#         38
  C:5265H         LINE#         39
  C:5265H         LINE#         40
  C:526BH         LINE#         41
  C:5271H         LINE#         42
  C:5271H         LINE#         43
  C:5281H         LINE#         44
  C:5281H         LINE#         45
  C:5281H         LINE#         46
  C:5281H         LINE#         47
  C:5287H         LINE#         48
  C:5287H         LINE#         49
  C:5287H         LINE#         50
  C:5287H         LINE#         51
  -------         ENDPROC       _DRAWFRAME
  -------         ENDMOD        TEXT_GRAPHICS_FUNCTIONS

  -------         MODULE        TXT_GRAPH
  C:4D39H         SEGMENT       ?PR?_DRAWSTRXRAM?TXT_GRAPH
  C:4F31H         SEGMENT       ?PR?_DRAWSTRBCK?TXT_GRAPH
  C:4C1EH         SEGMENT       ?PR?_DRAWLINE?TXT_GRAPH
  D:0036H         SEGMENT       ?DT?_DRAWLINE?TXT_GRAPH
  C:53D2H         SEGMENT       ?PR?_DRAWICON?TXT_GRAPH
  D:0008H         SEGMENT       ?DT?_DRAWICON?TXT_GRAPH
  D:0008H         PUBLIC        ?_DRAWICON?BYTE
  D:0036H         PUBLIC        ?_DRAWLINE?BYTE
  C:53D2H         PUBLIC        _DRAWICON
  C:4C1EH         PUBLIC        _DRAWLINE
  C:4D39H         PUBLIC        _DRAWSTRXRAM
  D:00E0H         SYMBOL        ACC
  D:00A2H         SYMBOL        AUXR1
  D:00F0H         SYMBOL        B
  D:0083H         SYMBOL        DPH
  D:0082H         SYMBOL        DPL
BL51 BANKED LINKER/LOCATER V4.02                                                      05/28/2008  17:48:13  PAGE 12


  C:4D38H         SYMBOL        DRAWLINEDONE
  C:4C72H         SYMBOL        DRAWLINEO2M1
  C:4C76H         SYMBOL        DRAWLINEO2M2
  C:4C7AH         SYMBOL        DRAWLINEO2M3
  C:4CB2H         SYMBOL        DRAWLINEQ1X
  C:4CB8H         SYMBOL        DRAWLINEQ1XL1
  C:4CD0H         SYMBOL        DRAWLINEQ1XS1
  C:4CD9H         SYMBOL        DRAWLINEQ1XS2
  C:4C8CH         SYMBOL        DRAWLINEQ1YL1
  C:4CA1H         SYMBOL        DRAWLINEQ1YS1
  C:4CDDH         SYMBOL        DRAWLINEQ4
  C:4D0FH         SYMBOL        DRAWLINEQ4X
  C:4D15H         SYMBOL        DRAWLINEQ4XL1
  C:4D2DH         SYMBOL        DRAWLINEQ4XS1
  C:4D36H         SYMBOL        DRAWLINEQ4XS2
  C:4CEAH         SYMBOL        DRAWLINEQ4YL1
  C:4CFFH         SYMBOL        DRAWLINEQ4YS1
  C:4C4BH         SYMBOL        DRAWLINEQC
  C:4F31H         SYMBOL        DRAWSTRBCK
  C:4F86H         SYMBOL        DRAWSTRBCKD
  C:500CH         SYMBOL        DRAWSTRBCKDE
  C:4FEEH         SYMBOL        DRAWSTRBCKDFL
  C:4FD0H         SYMBOL        DRAWSTRBCKDL
  C:500AH         SYMBOL        DRAWSTRBCKDS
  C:4F58H         SYMBOL        DRAWSTRBCKLL
  C:4FE0H         SYMBOL        DRAWSTRBCKNFL
  C:4D4FH         SYMBOL        DRAWSTRXRAMNI
  C:4D75H         SYMBOL        LCDWRTXT
  C:4E34H         SYMBOL        LCDWRTXTD
  C:4E30H         SYMBOL        LCDWRTXTDC
  C:4D7CH         SYMBOL        LCDWRTXTDN
  C:4E0AH         SYMBOL        LCDWRTXTL1
  C:4E25H         SYMBOL        LCDWRTXTL1S1
  C:4DE4H         SYMBOL        LCDWRTXTNL
  C:4E08H         SYMBOL        LCDWRTXTNNL
  N:0000H         SYMBOL        TXT_GRAPH
  C:544CH         SYMBOL        _DRAWICONE
  C:5416H         SYMBOL        _DRAWICONL1
  C:5414H         SYMBOL        _DRAWICONL2
  C:5431H         SYMBOL        _DRAWICONS1
  C:5414H         SYMBOL        _DRAWICONS2
  C:4D39H         LINE#         25
  C:4D3BH         LINE#         26
  C:4D3CH         LINE#         27
  C:4D3EH         LINE#         28
  C:4D40H         LINE#         29
  C:4D43H         LINE#         31
  C:4D45H         LINE#         32
  C:4D46H         LINE#         33
  C:4D49H         LINE#         34
  C:4D4AH         LINE#         35
  C:4D4CH         LINE#         36
  C:4D4FH         LINE#         37
  C:4D51H         LINE#         39
  C:4D52H         LINE#         40
  C:4D55H         LINE#         41
  C:4D56H         LINE#         42
BL51 BANKED LINKER/LOCATER V4.02                                                      05/28/2008  17:48:13  PAGE 13


  C:4D58H         LINE#         43
  C:4D5AH         LINE#         44
  C:4D5BH         LINE#         45
  C:4D5DH         LINE#         46
  C:4D5FH         LINE#         47
  C:4D60H         LINE#         48
  C:4D61H         LINE#         49
  C:4D62H         LINE#         50
  C:4D64H         LINE#         51
  C:4D65H         LINE#         52
  C:4D66H         LINE#         53
  C:4D68H         LINE#         54
  C:4D69H         LINE#         55
  C:4D6AH         LINE#         56
  C:4D6CH         LINE#         57
  C:4D6FH         LINE#         58
  C:4D72H         LINE#         60
  C:4D75H         LINE#         63
  C:4D76H         LINE#         64
  C:4D77H         LINE#         65
  C:4D79H         LINE#         66
  C:4D7CH         LINE#         67
  C:4D7EH         LINE#         68
  C:4D80H         LINE#         70
  C:4D83H         LINE#         71
  C:4D84H         LINE#         72
  C:4D85H         LINE#         73
  C:4D87H         LINE#         74
  C:4D89H         LINE#         75
  C:4D8AH         LINE#         76
  C:4D8CH         LINE#         77
  C:4D8EH         LINE#         78
  C:4D8FH         LINE#         79
  C:4D91H         LINE#         80
  C:4D93H         LINE#         81
  C:4D94H         LINE#         82
  C:4D97H         LINE#         83
  C:4D99H         LINE#         85
  C:4D9BH         LINE#         86
  C:4D9CH         LINE#         87
  C:4D9DH         LINE#         88
  C:4D9EH         LINE#         90
  C:4DA1H         LINE#         91
  C:4DA4H         LINE#         92
  C:4DA6H         LINE#         93
  C:4DA9H         LINE#         94
  C:4DABH         LINE#         95
  C:4DAEH         LINE#         96
  C:4DAFH         LINE#         97
  C:4DB2H         LINE#         98
  C:4DB3H         LINE#         99
  C:4DB4H         LINE#         101
  C:4DB6H         LINE#         103
  C:4DB8H         LINE#         104
  C:4DB9H         LINE#         105
  C:4DBAH         LINE#         106
  C:4DBBH         LINE#         107
BL51 BANKED LINKER/LOCATER V4.02                                                      05/28/2008  17:48:13  PAGE 14


  C:4DBDH         LINE#         108
  C:4DBFH         LINE#         109
  C:4DC1H         LINE#         110
  C:4DC3H         LINE#         111
  C:4DC5H         LINE#         112
  C:4DC7H         LINE#         113
  C:4DC9H         LINE#         114
  C:4DCCH         LINE#         115
  C:4DCDH         LINE#         116
  C:4DCFH         LINE#         117
  C:4DD1H         LINE#         118
  C:4DD3H         LINE#         119
  C:4DD5H         LINE#         121
  C:4DD7H         LINE#         123
  C:4DD8H         LINE#         124
  C:4DDAH         LINE#         125
  C:4DDBH         LINE#         126
  C:4DDDH         LINE#         127
  C:4DDFH         LINE#         128
  C:4DE0H         LINE#         129
  C:4DE2H         LINE#         130
  C:4DE4H         LINE#         132
  C:4DE6H         LINE#         133
  C:4DE7H         LINE#         134
  C:4DE9H         LINE#         135
  C:4DECH         LINE#         136
  C:4DEEH         LINE#         137
  C:4DF1H         LINE#         138
  C:4DF2H         LINE#         139
  C:4DF4H         LINE#         140
  C:4DF6H         LINE#         141
  C:4DF8H         LINE#         142
  C:4DFAH         LINE#         143
  C:4DFCH         LINE#         144
  C:4DFEH         LINE#         145
  C:4E00H         LINE#         146
  C:4E01H         LINE#         147
  C:4E04H         LINE#         148
  C:4E06H         LINE#         149
  C:4E08H         LINE#         152
  C:4E09H         LINE#         153
  C:4E0AH         LINE#         154
  C:4E0BH         LINE#         155
  C:4E0CH         LINE#         156
  C:4E0EH         LINE#         157
  C:4E0FH         LINE#         158
  C:4E10H         LINE#         159
  C:4E11H         LINE#         160
  C:4E13H         LINE#         161
  C:4E14H         LINE#         162
  C:4E15H         LINE#         163
  C:4E16H         LINE#         164
  C:4E17H         LINE#         165
  C:4E18H         LINE#         166
  C:4E1AH         LINE#         167
  C:4E1BH         LINE#         168
  C:4E1DH         LINE#         169
BL51 BANKED LINKER/LOCATER V4.02                                                      05/28/2008  17:48:13  PAGE 15


  C:4E1FH         LINE#         170
  C:4E21H         LINE#         171
  C:4E23H         LINE#         172
  C:4E25H         LINE#         173
  C:4E27H         LINE#         174
  C:4E29H         LINE#         176
  C:4E2BH         LINE#         177
  C:4E2DH         LINE#         178
  C:4E30H         LINE#         179
  C:4E32H         LINE#         180
  C:4E34H         LINE#         181
  C:4F31H         LINE#         191
  C:4F32H         LINE#         192
  C:4F35H         LINE#         193
  C:4F36H         LINE#         194
  C:4F38H         LINE#         195
  C:4F3AH         LINE#         196
  C:4F3BH         LINE#         197
  C:4F3DH         LINE#         198
  C:4F3FH         LINE#         199
  C:4F40H         LINE#         200
  C:4F41H         LINE#         201
  C:4F42H         LINE#         202
  C:4F44H         LINE#         203
  C:4F45H         LINE#         204
  C:4F46H         LINE#         205
  C:4F48H         LINE#         206
  C:4F49H         LINE#         207
  C:4F4AH         LINE#         208
  C:4F4CH         LINE#         209
  C:4F4DH         LINE#         210
  C:4F50H         LINE#         211
  C:4F53H         LINE#         213
  C:4F55H         LINE#         215
  C:4F58H         LINE#         217
  C:4F59H         LINE#         218
  C:4F5AH         LINE#         219
  C:4F5CH         LINE#         220
  C:4F5EH         LINE#         221
  C:4F60H         LINE#         223
  C:4F63H         LINE#         224
  C:4F64H         LINE#         225
  C:4F65H         LINE#         226
  C:4F67H         LINE#         227
  C:4F69H         LINE#         228
  C:4F6AH         LINE#         229
  C:4F6CH         LINE#         230
  C:4F6EH         LINE#         231
  C:4F6FH         LINE#         232
  C:4F71H         LINE#         233
  C:4F73H         LINE#         234
  C:4F74H         LINE#         235
  C:4F77H         LINE#         236
  C:4F79H         LINE#         238
  C:4F7BH         LINE#         239
  C:4F7CH         LINE#         240
  C:4F7DH         LINE#         241
BL51 BANKED LINKER/LOCATER V4.02                                                      05/28/2008  17:48:13  PAGE 16


  C:4F7EH         LINE#         242
  C:4F7FH         LINE#         243
  C:4F80H         LINE#         244
  C:4F82H         LINE#         245
  C:4F84H         LINE#         246
  C:4F86H         LINE#         248
  C:4F88H         LINE#         249
  C:4F8AH         LINE#         250
  C:4F8BH         LINE#         251
  C:4F8DH         LINE#         252
  C:4F8EH         LINE#         253
  C:4F90H         LINE#         254
  C:4F92H         LINE#         256
  C:4F94H         LINE#         257
  C:4F97H         LINE#         258
  C:4F98H         LINE#         259
  C:4F9AH         LINE#         260
  C:4F9CH         LINE#         261
  C:4F9EH         LINE#         262
  C:4FA0H         LINE#         263
  C:4FA2H         LINE#         266
  C:4FA4H         LINE#         267
  C:4FA6H         LINE#         268
  C:4FA7H         LINE#         269
  C:4FA8H         LINE#         270
  C:4FAAH         LINE#         271
  C:4FACH         LINE#         272
  C:4FADH         LINE#         273
  C:4FB0H         LINE#         274
  C:4FB1H         LINE#         275
  C:4FB2H         LINE#         276
  C:4FB4H         LINE#         277
  C:4FB7H         LINE#         278
  C:4FB9H         LINE#         279
  C:4FBCH         LINE#         280
  C:4FBDH         LINE#         281
  C:4FC0H         LINE#         282
  C:4FC1H         LINE#         283
  C:4FC2H         LINE#         285
  C:4FC4H         LINE#         286
  C:4FC5H         LINE#         287
  C:4FC7H         LINE#         288
  C:4FC9H         LINE#         289
  C:4FCBH         LINE#         290
  C:4FCDH         LINE#         292
  C:4FCEH         LINE#         293
  C:4FD0H         LINE#         295
  C:4FD2H         LINE#         296
  C:4FD4H         LINE#         297
  C:4FD6H         LINE#         299
  C:4FD7H         LINE#         300
  C:4FD8H         LINE#         301
  C:4FDAH         LINE#         302
  C:4FDCH         LINE#         303
  C:4FDDH         LINE#         304
  C:4FE0H         LINE#         306
  C:4FE2H         LINE#         307
BL51 BANKED LINKER/LOCATER V4.02                                                      05/28/2008  17:48:13  PAGE 17


  C:4FE4H         LINE#         308
  C:4FE6H         LINE#         309
  C:4FE8H         LINE#         310
  C:4FEAH         LINE#         311
  C:4FECH         LINE#         312
  C:4FEDH         LINE#         313
  C:4FEEH         LINE#         315
  C:4FEFH         LINE#         316
  C:4FF0H         LINE#         317
  C:4FF1H         LINE#         318
  C:4FF3H         LINE#         319
  C:4FF5H         LINE#         320
  C:4FF7H         LINE#         321
  C:4FF9H         LINE#         322
  C:4FFBH         LINE#         323
  C:4FFDH         LINE#         324
  C:4FFFH         LINE#         325
  C:5001H         LINE#         326
  C:5003H         LINE#         327
  C:5004H         LINE#         328
  C:5005H         LINE#         329
  C:5006H         LINE#         330
  C:5009H         LINE#         331
  C:500AH         LINE#         332
  C:500CH         LINE#         400
  C:4C1EH         LINE#         427
  C:4C1FH         LINE#         428
  C:4C20H         LINE#         429
  C:4C21H         LINE#         430
  C:4C23H         LINE#         431
  C:4C25H         LINE#         432
  C:4C26H         LINE#         433
  C:4C27H         LINE#         434
  C:4C28H         LINE#         435
  C:4C29H         LINE#         436
  C:4C2BH         LINE#         437
  C:4C2DH         LINE#         438
  C:4C2EH         LINE#         439
  C:4C2FH         LINE#         440
  C:4C30H         LINE#         441
  C:4C33H         LINE#         442
  C:4C34H         LINE#         443
  C:4C36H         LINE#         444
  C:4C37H         LINE#         445
  C:4C3AH         LINE#         446
  C:4C3BH         LINE#         453
  C:4C3CH         LINE#         454
  C:4C3DH         LINE#         455
  C:4C3EH         LINE#         456
  C:4C3FH         LINE#         457
  C:4C41H         LINE#         459
  C:4C42H         LINE#         460
  C:4C43H         LINE#         461
  C:4C44H         LINE#         462
  C:4C45H         LINE#         463
  C:4C46H         LINE#         464
  C:4C47H         LINE#         465
BL51 BANKED LINKER/LOCATER V4.02                                                      05/28/2008  17:48:13  PAGE 18


  C:4C48H         LINE#         466
  C:4C49H         LINE#         467
  C:4C4AH         LINE#         468
  C:4C4BH         LINE#         472
  C:4C4CH         LINE#         473
  C:4C4FH         LINE#         474
  C:4C50H         LINE#         475
  C:4C52H         LINE#         476
  C:4C54H         LINE#         477
  C:4C56H         LINE#         478
  C:4C58H         LINE#         479
  C:4C5AH         LINE#         480
  C:4C5CH         LINE#         481
  C:4C5DH         LINE#         482
  C:4C60H         LINE#         483
  C:4C61H         LINE#         484
  C:4C63H         LINE#         485
  C:4C65H         LINE#         486
  C:4C67H         LINE#         487
  C:4C69H         LINE#         489
  C:4C6BH         LINE#         490
  C:4C6DH         LINE#         491
  C:4C70H         LINE#         492
  C:4C72H         LINE#         493
  C:4C75H         LINE#         494
  C:4C76H         LINE#         495
  C:4C79H         LINE#         496
  C:4C7AH         LINE#         497
  C:4C7CH         LINE#         499
  C:4C7DH         LINE#         500
  C:4C7EH         LINE#         501
  C:4C7FH         LINE#         502
  C:4C81H         LINE#         504
  C:4C82H         LINE#         505
  C:4C83H         LINE#         506
  C:4C84H         LINE#         507
  C:4C86H         LINE#         509
  C:4C87H         LINE#         510
  C:4C88H         LINE#         511
  C:4C89H         LINE#         512
  C:4C8AH         LINE#         513
  C:4C8BH         LINE#         514
  C:4C8CH         LINE#         516
  C:4C8DH         LINE#         517
  C:4C8FH         LINE#         518
  C:4C90H         LINE#         519
  C:4C91H         LINE#         520
  C:4C92H         LINE#         521
  C:4C93H         LINE#         522
  C:4C94H         LINE#         523
  C:4C96H         LINE#         525
  C:4C97H         LINE#         526
  C:4C98H         LINE#         528
  C:4C9AH         LINE#         529
  C:4C9BH         LINE#         530
  C:4C9DH         LINE#         531
  C:4CA0H         LINE#         532
BL51 BANKED LINKER/LOCATER V4.02                                                      05/28/2008  17:48:13  PAGE 19


  C:4CA1H         LINE#         534
  C:4CA3H         LINE#         535
  C:4CA5H         LINE#         536
  C:4CA7H         LINE#         537
  C:4CA9H         LINE#         538
  C:4CABH         LINE#         539
  C:4CADH         LINE#         540
  C:4CAFH         LINE#         542
  C:4CB2H         LINE#         544
  C:4CB3H         LINE#         545
  C:4CB4H         LINE#         546
  C:4CB5H         LINE#         547
  C:4CB6H         LINE#         548
  C:4CB7H         LINE#         549
  C:4CB8H         LINE#         551
  C:4CB9H         LINE#         552
  C:4CBBH         LINE#         553
  C:4CBCH         LINE#         554
  C:4CBDH         LINE#         555
  C:4CBEH         LINE#         556
  C:4CBFH         LINE#         557
  C:4CC0H         LINE#         558
  C:4CC2H         LINE#         560
  C:4CC3H         LINE#         561
  C:4CC4H         LINE#         563
  C:4CC6H         LINE#         564
  C:4CC8H         LINE#         565
  C:4CCAH         LINE#         566
  C:4CCCH         LINE#         567
  C:4CCEH         LINE#         568
  C:4CD0H         LINE#         570
  C:4CD2H         LINE#         571
  C:4CD3H         LINE#         572
  C:4CD5H         LINE#         573
  C:4CD8H         LINE#         574
  C:4CD9H         LINE#         575
  C:4CDBH         LINE#         577
  C:4CDDH         LINE#         580
  C:4CDEH         LINE#         581
  C:4CDFH         LINE#         582
  C:4CE0H         LINE#         583
  C:4CE1H         LINE#         584
  C:4CE2H         LINE#         585
  C:4CE4H         LINE#         587
  C:4CE5H         LINE#         588
  C:4CE6H         LINE#         589
  C:4CE7H         LINE#         590
  C:4CE8H         LINE#         591
  C:4CE9H         LINE#         592
  C:4CEAH         LINE#         594
  C:4CEBH         LINE#         595
  C:4CEDH         LINE#         596
  C:4CEEH         LINE#         597
  C:4CEFH         LINE#         598
  C:4CF0H         LINE#         599
  C:4CF1H         LINE#         600
  C:4CF2H         LINE#         601
BL51 BANKED LINKER/LOCATER V4.02                                                      05/28/2008  17:48:13  PAGE 20


  C:4CF4H         LINE#         603
  C:4CF5H         LINE#         604
  C:4CF6H         LINE#         606
  C:4CF8H         LINE#         607
  C:4CF9H         LINE#         608
  C:4CFBH         LINE#         609
  C:4CFEH         LINE#         610
  C:4CFFH         LINE#         612
  C:4D01H         LINE#         613
  C:4D03H         LINE#         614
  C:4D05H         LINE#         615
  C:4D07H         LINE#         616
  C:4D09H         LINE#         617
  C:4D0BH         LINE#         618
  C:4D0DH         LINE#         620
  C:4D0FH         LINE#         622
  C:4D10H         LINE#         623
  C:4D11H         LINE#         624
  C:4D12H         LINE#         625
  C:4D13H         LINE#         626
  C:4D14H         LINE#         627
  C:4D15H         LINE#         629
  C:4D16H         LINE#         630
  C:4D18H         LINE#         631
  C:4D19H         LINE#         632
  C:4D1AH         LINE#         633
  C:4D1BH         LINE#         634
  C:4D1CH         LINE#         635
  C:4D1DH         LINE#         636
  C:4D1FH         LINE#         638
  C:4D20H         LINE#         639
  C:4D21H         LINE#         641
  C:4D23H         LINE#         642
  C:4D25H         LINE#         643
  C:4D27H         LINE#         644
  C:4D29H         LINE#         645
  C:4D2BH         LINE#         646
  C:4D2DH         LINE#         648
  C:4D2FH         LINE#         649
  C:4D30H         LINE#         650
  C:4D32H         LINE#         651
  C:4D35H         LINE#         652
  C:4D36H         LINE#         653
  C:4D38H         LINE#         657
  C:53D2H         LINE#         673
  C:53D3H         LINE#         674
  C:53D6H         LINE#         675
  C:53D8H         LINE#         676
  C:53D9H         LINE#         677
  C:53DCH         LINE#         678
  C:53DDH         LINE#         679
  C:53DEH         LINE#         680
  C:53E0H         LINE#         681
  C:53E2H         LINE#         682
  C:53E3H         LINE#         683
  C:53E4H         LINE#         684
  C:53E5H         LINE#         685
BL51 BANKED LINKER/LOCATER V4.02                                                      05/28/2008  17:48:13  PAGE 21


  C:53E7H         LINE#         686
  C:53E9H         LINE#         688
  C:53EBH         LINE#         689
  C:53EDH         LINE#         690
  C:53EEH         LINE#         691
  C:53EFH         LINE#         692
  C:53F0H         LINE#         693
  C:53F1H         LINE#         694
  C:53F2H         LINE#         695
  C:53F3H         LINE#         696
  C:53F4H         LINE#         697
  C:53F6H         LINE#         698
  C:53F7H         LINE#         699
  C:53F9H         LINE#         700
  C:53FBH         LINE#         701
  C:53FDH         LINE#         702
  C:53FFH         LINE#         703
  C:5401H         LINE#         704
  C:5403H         LINE#         705
  C:5405H         LINE#         706
  C:5407H         LINE#         707
  C:5409H         LINE#         708
  C:540AH         LINE#         709
  C:540DH         LINE#         710
  C:540EH         LINE#         711
  C:5410H         LINE#         712
  C:5412H         LINE#         713
  C:5414H         LINE#         715
  C:5416H         LINE#         716
  C:5418H         LINE#         717
  C:541AH         LINE#         718
  C:541DH         LINE#         719
  C:5420H         LINE#         720
  C:5421H         LINE#         721
  C:5422H         LINE#         722
  C:5423H         LINE#         723
  C:5426H         LINE#         724
  C:5429H         LINE#         725
  C:542BH         LINE#         726
  C:542DH         LINE#         727
  C:542EH         LINE#         728
  C:542FH         LINE#         729
  C:5431H         LINE#         730
  C:5432H         LINE#         731
  C:5434H         LINE#         732
  C:5436H         LINE#         733
  C:5438H         LINE#         734
  C:543AH         LINE#         735
  C:543CH         LINE#         736
  C:543EH         LINE#         737
  C:5440H         LINE#         738
  C:5442H         LINE#         739
  C:5444H         LINE#         740
  C:5446H         LINE#         741
  C:5448H         LINE#         742
  C:544AH         LINE#         743
  C:544CH         LINE#         744
BL51 BANKED LINKER/LOCATER V4.02                                                      05/28/2008  17:48:13  PAGE 22


  -------         ENDMOD        TXT_GRAPH

  -------         MODULE        FONTS
  C:0026H         SEGMENT       CODESEG
  C:00CFH         PUBLIC        FONTLIST
  C:00DBH         SYMBOL        FONT08PX
  C:060EH         SYMBOL        FONT08PX_123
  C:0617H         SYMBOL        FONT08PX_124
  C:0620H         SYMBOL        FONT08PX_125
  C:0629H         SYMBOL        FONT08PX_126
  C:02DBH         SYMBOL        FONT08PX_32
  C:02E4H         SYMBOL        FONT08PX_33
  C:02EDH         SYMBOL        FONT08PX_34
  C:02F6H         SYMBOL        FONT08PX_35
  C:02FFH         SYMBOL        FONT08PX_36
  C:0308H         SYMBOL        FONT08PX_37
  C:0311H         SYMBOL        FONT08PX_38
  C:031AH         SYMBOL        FONT08PX_39
  C:0323H         SYMBOL        FONT08PX_40
  C:032CH         SYMBOL        FONT08PX_41
  C:0335H         SYMBOL        FONT08PX_42
  C:033EH         SYMBOL        FONT08PX_43
  C:0347H         SYMBOL        FONT08PX_44
  C:0350H         SYMBOL        FONT08PX_45
  C:0359H         SYMBOL        FONT08PX_46
  C:0362H         SYMBOL        FONT08PX_47
  C:03C5H         SYMBOL        FONT08PX_58
  C:03CEH         SYMBOL        FONT08PX_59
  C:03D7H         SYMBOL        FONT08PX_60
  C:03E0H         SYMBOL        FONT08PX_61
  C:03E9H         SYMBOL        FONT08PX_62
  C:03F2H         SYMBOL        FONT08PX_63
  C:03FBH         SYMBOL        FONT08PX_64
  C:04EEH         SYMBOL        FONT08PX_91
  C:04F7H         SYMBOL        FONT08PX_92
  C:0500H         SYMBOL        FONT08PX_93
  C:0509H         SYMBOL        FONT08PX_94
  C:0512H         SYMBOL        FONT08PX_95
  C:051BH         SYMBOL        FONT08PX_96
  C:0749H         SYMBOL        FONT08PX_BLANK
  C:0524H         SYMBOL        FONT08PX_LA
  C:06D4H         SYMBOL        FONT08PX_LAA
  C:052DH         SYMBOL        FONT08PX_LB
  C:0536H         SYMBOL        FONT08PX_LC
  C:06DDH         SYMBOL        FONT08PX_LCH
  C:053FH         SYMBOL        FONT08PX_LD
  C:070AH         SYMBOL        FONT08PX_LDH
  C:0548H         SYMBOL        FONT08PX_LE
  C:06E6H         SYMBOL        FONT08PX_LEE
  C:06F8H         SYMBOL        FONT08PX_LEH
  C:06EFH         SYMBOL        FONT08PX_LEP
  C:0551H         SYMBOL        FONT08PX_LF
  C:055AH         SYMBOL        FONT08PX_LG
  C:0563H         SYMBOL        FONT08PX_LH
  C:056CH         SYMBOL        FONT08PX_LI
  C:0701H         SYMBOL        FONT08PX_LII
  C:0575H         SYMBOL        FONT08PX_LJ
BL51 BANKED LINKER/LOCATER V4.02                                                      05/28/2008  17:48:13  PAGE 23


  C:057EH         SYMBOL        FONT08PX_LK
  C:0587H         SYMBOL        FONT08PX_LL
  C:0590H         SYMBOL        FONT08PX_LM
  C:0599H         SYMBOL        FONT08PX_LN
  C:0713H         SYMBOL        FONT08PX_LNH
  C:05A2H         SYMBOL        FONT08PX_LO
  C:071CH         SYMBOL        FONT08PX_LOO
  C:05ABH         SYMBOL        FONT08PX_LP
  C:05B4H         SYMBOL        FONT08PX_LQ
  C:05BDH         SYMBOL        FONT08PX_LR
  C:0725H         SYMBOL        FONT08PX_LRH
  C:05C6H         SYMBOL        FONT08PX_LS
  C:064DH         SYMBOL        FONT08PX_LSH
  C:05CFH         SYMBOL        FONT08PX_LT
  C:0656H         SYMBOL        FONT08PX_LTH
  C:05D8H         SYMBOL        FONT08PX_LU
  C:072EH         SYMBOL        FONT08PX_LUK
  C:0737H         SYMBOL        FONT08PX_LUU
  C:05E1H         SYMBOL        FONT08PX_LV
  C:05EAH         SYMBOL        FONT08PX_LW
  C:05F3H         SYMBOL        FONT08PX_LX
  C:05FCH         SYMBOL        FONT08PX_LY
  C:0740H         SYMBOL        FONT08PX_LYY
  C:0605H         SYMBOL        FONT08PX_LZ
  C:065FH         SYMBOL        FONT08PX_LZH
  C:036BH         SYMBOL        FONT08PX_N0
  C:0374H         SYMBOL        FONT08PX_N1
  C:037DH         SYMBOL        FONT08PX_N2
  C:0386H         SYMBOL        FONT08PX_N3
  C:038FH         SYMBOL        FONT08PX_N4
  C:0398H         SYMBOL        FONT08PX_N5
  C:03A1H         SYMBOL        FONT08PX_N6
  C:03AAH         SYMBOL        FONT08PX_N7
  C:03B3H         SYMBOL        FONT08PX_N8
  C:03BCH         SYMBOL        FONT08PX_N9
  C:0404H         SYMBOL        FONT08PX_UA
  C:0668H         SYMBOL        FONT08PX_UAA
  C:040DH         SYMBOL        FONT08PX_UB
  C:0416H         SYMBOL        FONT08PX_UC
  C:0671H         SYMBOL        FONT08PX_UCH
  C:041FH         SYMBOL        FONT08PX_UD
  C:0695H         SYMBOL        FONT08PX_UDH
  C:0428H         SYMBOL        FONT08PX_UE
  C:067AH         SYMBOL        FONT08PX_UEE
  C:0683H         SYMBOL        FONT08PX_UEH
  C:0431H         SYMBOL        FONT08PX_UF
  C:043AH         SYMBOL        FONT08PX_UG
  C:0443H         SYMBOL        FONT08PX_UH
  C:044CH         SYMBOL        FONT08PX_UI
  C:068CH         SYMBOL        FONT08PX_UII
  C:0455H         SYMBOL        FONT08PX_UJ
  C:045EH         SYMBOL        FONT08PX_UK
  C:0467H         SYMBOL        FONT08PX_UL
  C:0470H         SYMBOL        FONT08PX_UM
  C:0479H         SYMBOL        FONT08PX_UN
  C:069EH         SYMBOL        FONT08PX_UNH
  C:0482H         SYMBOL        FONT08PX_UO
BL51 BANKED LINKER/LOCATER V4.02                                                      05/28/2008  17:48:13  PAGE 24


  C:06A7H         SYMBOL        FONT08PX_UOO
  C:048BH         SYMBOL        FONT08PX_UP
  C:0494H         SYMBOL        FONT08PX_UQ
  C:049DH         SYMBOL        FONT08PX_UR
  C:06B0H         SYMBOL        FONT08PX_URH
  C:04A6H         SYMBOL        FONT08PX_US
  C:0632H         SYMBOL        FONT08PX_USH
  C:04AFH         SYMBOL        FONT08PX_UT
  C:063BH         SYMBOL        FONT08PX_UTH
  C:04B8H         SYMBOL        FONT08PX_UU
  C:06B9H         SYMBOL        FONT08PX_UUK
  C:06C2H         SYMBOL        FONT08PX_UUU
  C:04C1H         SYMBOL        FONT08PX_UV
  C:04CAH         SYMBOL        FONT08PX_UW
  C:04D3H         SYMBOL        FONT08PX_UX
  C:04DCH         SYMBOL        FONT08PX_UY
  C:06CBH         SYMBOL        FONT08PX_UYY
  C:04E5H         SYMBOL        FONT08PX_UZ
  C:0644H         SYMBOL        FONT08PX_UZH
  C:0752H         SYMBOL        FONT12PX
  C:0DE4H         SYMBOL        FONT12PX_123
  C:0DF1H         SYMBOL        FONT12PX_124
  C:0DFEH         SYMBOL        FONT12PX_125
  C:0E0BH         SYMBOL        FONT12PX_126
  C:095FH         SYMBOL        FONT12PX_33
  C:096CH         SYMBOL        FONT12PX_34
  C:0979H         SYMBOL        FONT12PX_35
  C:0986H         SYMBOL        FONT12PX_36
  C:0993H         SYMBOL        FONT12PX_37
  C:09A0H         SYMBOL        FONT12PX_38
  C:09ADH         SYMBOL        FONT12PX_39
  C:09BAH         SYMBOL        FONT12PX_40
  C:09C7H         SYMBOL        FONT12PX_41
  C:09D4H         SYMBOL        FONT12PX_42
  C:09E1H         SYMBOL        FONT12PX_43
  C:09EEH         SYMBOL        FONT12PX_44
  C:09FBH         SYMBOL        FONT12PX_45
  C:0A08H         SYMBOL        FONT12PX_46
  C:0A15H         SYMBOL        FONT12PX_47
  C:0AA4H         SYMBOL        FONT12PX_58
  C:0AB1H         SYMBOL        FONT12PX_59
  C:0ABEH         SYMBOL        FONT12PX_60
  C:0ACBH         SYMBOL        FONT12PX_61
  C:0AD8H         SYMBOL        FONT12PX_62
  C:0AE5H         SYMBOL        FONT12PX_63
  C:0C44H         SYMBOL        FONT12PX_91
  C:0C51H         SYMBOL        FONT12PX_92
  C:0C5EH         SYMBOL        FONT12PX_93
  C:0C6BH         SYMBOL        FONT12PX_94
  C:0C78H         SYMBOL        FONT12PX_95
  C:0C85H         SYMBOL        FONT12PX_96
  C:0F91H         SYMBOL        FONT12PX_BLANK
  C:0C92H         SYMBOL        FONT12PX_LA
  C:0EF5H         SYMBOL        FONT12PX_LAA
  C:0C9FH         SYMBOL        FONT12PX_LB
  C:0CACH         SYMBOL        FONT12PX_LC
  C:0F02H         SYMBOL        FONT12PX_LCH
BL51 BANKED LINKER/LOCATER V4.02                                                      05/28/2008  17:48:13  PAGE 25


  C:0CB9H         SYMBOL        FONT12PX_LD
  C:0F36H         SYMBOL        FONT12PX_LDH
  C:0CC6H         SYMBOL        FONT12PX_LE
  C:0F0FH         SYMBOL        FONT12PX_LEE
  C:0F1CH         SYMBOL        FONT12PX_LEH
  C:0CD3H         SYMBOL        FONT12PX_LF
  C:0CE0H         SYMBOL        FONT12PX_LG
  C:0CEDH         SYMBOL        FONT12PX_LH
  C:0CFAH         SYMBOL        FONT12PX_LI
  C:0F29H         SYMBOL        FONT12PX_LII
  C:0D07H         SYMBOL        FONT12PX_LJ
  C:0D14H         SYMBOL        FONT12PX_LK
  C:0D21H         SYMBOL        FONT12PX_LL
  C:0D2EH         SYMBOL        FONT12PX_LM
  C:0D3BH         SYMBOL        FONT12PX_LN
  C:0F43H         SYMBOL        FONT12PX_LNH
  C:0D48H         SYMBOL        FONT12PX_LO
  C:0F50H         SYMBOL        FONT12PX_LOO
  C:0D55H         SYMBOL        FONT12PX_LP
  C:0D62H         SYMBOL        FONT12PX_LQ
  C:0D6FH         SYMBOL        FONT12PX_LR
  C:0F5DH         SYMBOL        FONT12PX_LRH
  C:0D7CH         SYMBOL        FONT12PX_LS
  C:0E3FH         SYMBOL        FONT12PX_LSH
  C:0D89H         SYMBOL        FONT12PX_LT
  C:0E4CH         SYMBOL        FONT12PX_LTH
  C:0D96H         SYMBOL        FONT12PX_LU
  C:0F6AH         SYMBOL        FONT12PX_LUK
  C:0F77H         SYMBOL        FONT12PX_LUU
  C:0DA3H         SYMBOL        FONT12PX_LV
  C:0DB0H         SYMBOL        FONT12PX_LW
  C:0DBDH         SYMBOL        FONT12PX_LX
  C:0DCAH         SYMBOL        FONT12PX_LY
  C:0F84H         SYMBOL        FONT12PX_LYY
  C:0DD7H         SYMBOL        FONT12PX_LZ
  C:0E59H         SYMBOL        FONT12PX_LZH
  C:0A22H         SYMBOL        FONT12PX_N0
  C:0A2FH         SYMBOL        FONT12PX_N1
  C:0A3CH         SYMBOL        FONT12PX_N2
  C:0A49H         SYMBOL        FONT12PX_N3
  C:0A56H         SYMBOL        FONT12PX_N4
  C:0A63H         SYMBOL        FONT12PX_N5
  C:0A70H         SYMBOL        FONT12PX_N6
  C:0A7DH         SYMBOL        FONT12PX_N7
  C:0A8AH         SYMBOL        FONT12PX_N8
  C:0A97H         SYMBOL        FONT12PX_N9
  C:0952H         SYMBOL        FONT12PX_SPACE
  C:0AF2H         SYMBOL        FONT12PX_UA
  C:0E66H         SYMBOL        FONT12PX_UAA
  C:0AFFH         SYMBOL        FONT12PX_UB
  C:0B0CH         SYMBOL        FONT12PX_UC
  C:0B19H         SYMBOL        FONT12PX_UD
  C:0E9AH         SYMBOL        FONT12PX_UDH
  C:0B26H         SYMBOL        FONT12PX_UE
  C:0E73H         SYMBOL        FONT12PX_UEE
  C:0E80H         SYMBOL        FONT12PX_UEH
  C:0B33H         SYMBOL        FONT12PX_UF
BL51 BANKED LINKER/LOCATER V4.02                                                      05/28/2008  17:48:13  PAGE 26


  C:0B40H         SYMBOL        FONT12PX_UG
  C:0B4DH         SYMBOL        FONT12PX_UH
  C:0B5AH         SYMBOL        FONT12PX_UI
  C:0E8DH         SYMBOL        FONT12PX_UII
  C:0B67H         SYMBOL        FONT12PX_UJ
  C:0B74H         SYMBOL        FONT12PX_UK
  C:0B81H         SYMBOL        FONT12PX_UL
  C:0B8EH         SYMBOL        FONT12PX_UM
  C:0B9BH         SYMBOL        FONT12PX_UN
  C:0EA7H         SYMBOL        FONT12PX_UNH
  C:0BA8H         SYMBOL        FONT12PX_UO
  C:0EB4H         SYMBOL        FONT12PX_UOO
  C:0BB5H         SYMBOL        FONT12PX_UP
  C:0BC2H         SYMBOL        FONT12PX_UQ
  C:0BCFH         SYMBOL        FONT12PX_UR
  C:0EC1H         SYMBOL        FONT12PX_URH
  C:0BDCH         SYMBOL        FONT12PX_US
  C:0E18H         SYMBOL        FONT12PX_USH
  C:0BE9H         SYMBOL        FONT12PX_UT
  C:0E25H         SYMBOL        FONT12PX_UTH
  C:0BF6H         SYMBOL        FONT12PX_UU
  C:0ECEH         SYMBOL        FONT12PX_UUK
  C:0EDBH         SYMBOL        FONT12PX_UUU
  C:0C03H         SYMBOL        FONT12PX_UV
  C:0C10H         SYMBOL        FONT12PX_UW
  C:0C1DH         SYMBOL        FONT12PX_UX
  C:0C2AH         SYMBOL        FONT12PX_UY
  C:0EE8H         SYMBOL        FONT12PX_UYY
  C:0C37H         SYMBOL        FONT12PX_UZ
  C:0E32H         SYMBOL        FONT12PX_UZH
  C:0F9EH         SYMBOL        FONT16PX
  C:1DE7H         SYMBOL        FONT16PXBOLD
  C:246BH         SYMBOL        FONT16PXBOLD_100
  C:247CH         SYMBOL        FONT16PXBOLD_101
  C:248DH         SYMBOL        FONT16PXBOLD_102
  C:249EH         SYMBOL        FONT16PXBOLD_103
  C:24AFH         SYMBOL        FONT16PXBOLD_104
  C:24C0H         SYMBOL        FONT16PXBOLD_105
  C:24D1H         SYMBOL        FONT16PXBOLD_106
  C:24E2H         SYMBOL        FONT16PXBOLD_107
  C:24F3H         SYMBOL        FONT16PXBOLD_108
  C:2504H         SYMBOL        FONT16PXBOLD_109
  C:2515H         SYMBOL        FONT16PXBOLD_110
  C:2526H         SYMBOL        FONT16PXBOLD_111
  C:2537H         SYMBOL        FONT16PXBOLD_112
  C:2548H         SYMBOL        FONT16PXBOLD_113
  C:2559H         SYMBOL        FONT16PXBOLD_114
  C:256AH         SYMBOL        FONT16PXBOLD_115
  C:257BH         SYMBOL        FONT16PXBOLD_116
  C:258CH         SYMBOL        FONT16PXBOLD_117
  C:259DH         SYMBOL        FONT16PXBOLD_118
  C:25AEH         SYMBOL        FONT16PXBOLD_119
  C:25BFH         SYMBOL        FONT16PXBOLD_120
  C:25D0H         SYMBOL        FONT16PXBOLD_121
  C:25E1H         SYMBOL        FONT16PXBOLD_122
  C:25F2H         SYMBOL        FONT16PXBOLD_123
  C:2603H         SYMBOL        FONT16PXBOLD_124
BL51 BANKED LINKER/LOCATER V4.02                                                      05/28/2008  17:48:13  PAGE 27


  C:2614H         SYMBOL        FONT16PXBOLD_125
  C:2625H         SYMBOL        FONT16PXBOLD_126
  C:2636H         SYMBOL        FONT16PXBOLD_138
  C:2647H         SYMBOL        FONT16PXBOLD_141
  C:2658H         SYMBOL        FONT16PXBOLD_142
  C:2669H         SYMBOL        FONT16PXBOLD_154
  C:267AH         SYMBOL        FONT16PXBOLD_157
  C:268BH         SYMBOL        FONT16PXBOLD_158
  C:269CH         SYMBOL        FONT16PXBOLD_167
  C:26ADH         SYMBOL        FONT16PXBOLD_169
  C:26BEH         SYMBOL        FONT16PXBOLD_193
  C:26CFH         SYMBOL        FONT16PXBOLD_200
  C:26E0H         SYMBOL        FONT16PXBOLD_201
  C:26F1H         SYMBOL        FONT16PXBOLD_204
  C:2702H         SYMBOL        FONT16PXBOLD_205
  C:2713H         SYMBOL        FONT16PXBOLD_207
  C:2724H         SYMBOL        FONT16PXBOLD_210
  C:2735H         SYMBOL        FONT16PXBOLD_211
  C:2746H         SYMBOL        FONT16PXBOLD_216
  C:2757H         SYMBOL        FONT16PXBOLD_217
  C:2768H         SYMBOL        FONT16PXBOLD_218
  C:2779H         SYMBOL        FONT16PXBOLD_221
  C:278AH         SYMBOL        FONT16PXBOLD_225
  C:279BH         SYMBOL        FONT16PXBOLD_232
  C:27ACH         SYMBOL        FONT16PXBOLD_233
  C:27BDH         SYMBOL        FONT16PXBOLD_236
  C:27CEH         SYMBOL        FONT16PXBOLD_237
  C:27DFH         SYMBOL        FONT16PXBOLD_239
  C:27F0H         SYMBOL        FONT16PXBOLD_242
  C:2801H         SYMBOL        FONT16PXBOLD_243
  C:2812H         SYMBOL        FONT16PXBOLD_248
  C:2823H         SYMBOL        FONT16PXBOLD_249
  C:2834H         SYMBOL        FONT16PXBOLD_250
  C:2845H         SYMBOL        FONT16PXBOLD_253
  C:1FE7H         SYMBOL        FONT16PXBOLD_32
  C:1FF8H         SYMBOL        FONT16PXBOLD_33
  C:2009H         SYMBOL        FONT16PXBOLD_34
  C:201AH         SYMBOL        FONT16PXBOLD_35
  C:202BH         SYMBOL        FONT16PXBOLD_36
  C:203CH         SYMBOL        FONT16PXBOLD_37
  C:204DH         SYMBOL        FONT16PXBOLD_38
  C:205EH         SYMBOL        FONT16PXBOLD_39
  C:206FH         SYMBOL        FONT16PXBOLD_40
  C:2080H         SYMBOL        FONT16PXBOLD_41
  C:2091H         SYMBOL        FONT16PXBOLD_42
  C:20A2H         SYMBOL        FONT16PXBOLD_43
  C:20B3H         SYMBOL        FONT16PXBOLD_44
  C:20C4H         SYMBOL        FONT16PXBOLD_45
  C:20D5H         SYMBOL        FONT16PXBOLD_46
  C:20E6H         SYMBOL        FONT16PXBOLD_47
  C:20F7H         SYMBOL        FONT16PXBOLD_48
  C:2108H         SYMBOL        FONT16PXBOLD_49
  C:2119H         SYMBOL        FONT16PXBOLD_50
  C:212AH         SYMBOL        FONT16PXBOLD_51
  C:213BH         SYMBOL        FONT16PXBOLD_52
  C:214CH         SYMBOL        FONT16PXBOLD_53
  C:215DH         SYMBOL        FONT16PXBOLD_54
BL51 BANKED LINKER/LOCATER V4.02                                                      05/28/2008  17:48:13  PAGE 28


  C:216EH         SYMBOL        FONT16PXBOLD_55
  C:217FH         SYMBOL        FONT16PXBOLD_56
  C:2190H         SYMBOL        FONT16PXBOLD_57
  C:21A1H         SYMBOL        FONT16PXBOLD_58
  C:21B2H         SYMBOL        FONT16PXBOLD_59
  C:21C3H         SYMBOL        FONT16PXBOLD_60
  C:21D4H         SYMBOL        FONT16PXBOLD_61
  C:21E5H         SYMBOL        FONT16PXBOLD_62
  C:21F6H         SYMBOL        FONT16PXBOLD_63
  C:2207H         SYMBOL        FONT16PXBOLD_64
  C:2218H         SYMBOL        FONT16PXBOLD_65
  C:2229H         SYMBOL        FONT16PXBOLD_66
  C:223AH         SYMBOL        FONT16PXBOLD_67
  C:224BH         SYMBOL        FONT16PXBOLD_68
  C:225CH         SYMBOL        FONT16PXBOLD_69
  C:226DH         SYMBOL        FONT16PXBOLD_70
  C:227EH         SYMBOL        FONT16PXBOLD_71
  C:228FH         SYMBOL        FONT16PXBOLD_72
  C:22A0H         SYMBOL        FONT16PXBOLD_73
  C:22B1H         SYMBOL        FONT16PXBOLD_74
  C:22C2H         SYMBOL        FONT16PXBOLD_75
  C:22D3H         SYMBOL        FONT16PXBOLD_76
  C:22E4H         SYMBOL        FONT16PXBOLD_77
  C:22F5H         SYMBOL        FONT16PXBOLD_78
  C:2306H         SYMBOL        FONT16PXBOLD_79
  C:2317H         SYMBOL        FONT16PXBOLD_80
  C:2328H         SYMBOL        FONT16PXBOLD_81
  C:2339H         SYMBOL        FONT16PXBOLD_82
  C:234AH         SYMBOL        FONT16PXBOLD_83
  C:235BH         SYMBOL        FONT16PXBOLD_84
  C:236CH         SYMBOL        FONT16PXBOLD_85
  C:237DH         SYMBOL        FONT16PXBOLD_86
  C:238EH         SYMBOL        FONT16PXBOLD_87
  C:239FH         SYMBOL        FONT16PXBOLD_88
  C:23B0H         SYMBOL        FONT16PXBOLD_89
  C:23C1H         SYMBOL        FONT16PXBOLD_90
  C:23D2H         SYMBOL        FONT16PXBOLD_91
  C:23E3H         SYMBOL        FONT16PXBOLD_92
  C:23F4H         SYMBOL        FONT16PXBOLD_93
  C:2405H         SYMBOL        FONT16PXBOLD_94
  C:2416H         SYMBOL        FONT16PXBOLD_95
  C:2427H         SYMBOL        FONT16PXBOLD_96
  C:2438H         SYMBOL        FONT16PXBOLD_97
  C:2449H         SYMBOL        FONT16PXBOLD_98
  C:245AH         SYMBOL        FONT16PXBOLD_99
  C:2856H         SYMBOL        FONT16PXBOLD_BLANK
  C:1622H         SYMBOL        FONT16PX_100
  C:1633H         SYMBOL        FONT16PX_101
  C:1644H         SYMBOL        FONT16PX_102
  C:1655H         SYMBOL        FONT16PX_103
  C:1666H         SYMBOL        FONT16PX_104
  C:1677H         SYMBOL        FONT16PX_105
  C:1688H         SYMBOL        FONT16PX_106
  C:1699H         SYMBOL        FONT16PX_107
  C:16AAH         SYMBOL        FONT16PX_108
  C:16BBH         SYMBOL        FONT16PX_109
  C:16CCH         SYMBOL        FONT16PX_110
BL51 BANKED LINKER/LOCATER V4.02                                                      05/28/2008  17:48:13  PAGE 29


  C:16DDH         SYMBOL        FONT16PX_111
  C:16EEH         SYMBOL        FONT16PX_112
  C:16FFH         SYMBOL        FONT16PX_113
  C:1710H         SYMBOL        FONT16PX_114
  C:1721H         SYMBOL        FONT16PX_115
  C:1732H         SYMBOL        FONT16PX_116
  C:1743H         SYMBOL        FONT16PX_117
  C:1754H         SYMBOL        FONT16PX_118
  C:1765H         SYMBOL        FONT16PX_119
  C:1776H         SYMBOL        FONT16PX_120
  C:1787H         SYMBOL        FONT16PX_121
  C:1798H         SYMBOL        FONT16PX_122
  C:17A9H         SYMBOL        FONT16PX_123
  C:17BAH         SYMBOL        FONT16PX_124
  C:17CBH         SYMBOL        FONT16PX_125
  C:17DCH         SYMBOL        FONT16PX_126
  C:17EDH         SYMBOL        FONT16PX_138
  C:17FEH         SYMBOL        FONT16PX_139
  C:180FH         SYMBOL        FONT16PX_140
  C:1820H         SYMBOL        FONT16PX_141
  C:1831H         SYMBOL        FONT16PX_142
  C:1842H         SYMBOL        FONT16PX_143
  C:1853H         SYMBOL        FONT16PX_154
  C:1864H         SYMBOL        FONT16PX_156
  C:1875H         SYMBOL        FONT16PX_157
  C:1886H         SYMBOL        FONT16PX_158
  C:1897H         SYMBOL        FONT16PX_159
  C:18A8H         SYMBOL        FONT16PX_161
  C:18B9H         SYMBOL        FONT16PX_163
  C:18CAH         SYMBOL        FONT16PX_165
  C:18DBH         SYMBOL        FONT16PX_167
  C:18ECH         SYMBOL        FONT16PX_168
  C:18FDH         SYMBOL        FONT16PX_169
  C:190EH         SYMBOL        FONT16PX_170
  C:191FH         SYMBOL        FONT16PX_175
  C:1930H         SYMBOL        FONT16PX_176
  C:1941H         SYMBOL        FONT16PX_179
  C:1952H         SYMBOL        FONT16PX_180
  C:1963H         SYMBOL        FONT16PX_185
  C:1974H         SYMBOL        FONT16PX_186
  C:1985H         SYMBOL        FONT16PX_188
  C:1996H         SYMBOL        FONT16PX_190
  C:19A7H         SYMBOL        FONT16PX_191
  C:19B8H         SYMBOL        FONT16PX_192
  C:19C9H         SYMBOL        FONT16PX_193
  C:19DAH         SYMBOL        FONT16PX_194
  C:19EBH         SYMBOL        FONT16PX_195
  C:19FCH         SYMBOL        FONT16PX_196
  C:1A0DH         SYMBOL        FONT16PX_197
  C:1A1EH         SYMBOL        FONT16PX_198
  C:1A2FH         SYMBOL        FONT16PX_199
  C:1A40H         SYMBOL        FONT16PX_200
  C:1A51H         SYMBOL        FONT16PX_201
  C:1A62H         SYMBOL        FONT16PX_202
  C:1A73H         SYMBOL        FONT16PX_203
  C:1A84H         SYMBOL        FONT16PX_204
  C:1A95H         SYMBOL        FONT16PX_205
BL51 BANKED LINKER/LOCATER V4.02                                                      05/28/2008  17:48:13  PAGE 30


  C:1AA6H         SYMBOL        FONT16PX_206
  C:1AB7H         SYMBOL        FONT16PX_207
  C:1AC8H         SYMBOL        FONT16PX_208
  C:1AD9H         SYMBOL        FONT16PX_209
  C:1AEAH         SYMBOL        FONT16PX_210
  C:1AFBH         SYMBOL        FONT16PX_211
  C:1B0CH         SYMBOL        FONT16PX_212
  C:1B1DH         SYMBOL        FONT16PX_213
  C:1B2EH         SYMBOL        FONT16PX_214
  C:1B3FH         SYMBOL        FONT16PX_215
  C:1B50H         SYMBOL        FONT16PX_216
  C:1B61H         SYMBOL        FONT16PX_217
  C:1B72H         SYMBOL        FONT16PX_218
  C:1B83H         SYMBOL        FONT16PX_219
  C:1B94H         SYMBOL        FONT16PX_220
  C:1BA5H         SYMBOL        FONT16PX_221
  C:1BB6H         SYMBOL        FONT16PX_222
  C:1BC7H         SYMBOL        FONT16PX_223
  C:1BD8H         SYMBOL        FONT16PX_224
  C:1BE9H         SYMBOL        FONT16PX_225
  C:1BFAH         SYMBOL        FONT16PX_226
  C:1C0BH         SYMBOL        FONT16PX_227
  C:1C1CH         SYMBOL        FONT16PX_228
  C:1C2DH         SYMBOL        FONT16PX_229
  C:1C3EH         SYMBOL        FONT16PX_230
  C:1C4FH         SYMBOL        FONT16PX_231
  C:1C60H         SYMBOL        FONT16PX_232
  C:1C71H         SYMBOL        FONT16PX_233
  C:1C82H         SYMBOL        FONT16PX_234
  C:1C93H         SYMBOL        FONT16PX_235
  C:1CA4H         SYMBOL        FONT16PX_236
  C:1CB5H         SYMBOL        FONT16PX_237
  C:1CC6H         SYMBOL        FONT16PX_238
  C:1CD7H         SYMBOL        FONT16PX_239
  C:1CE8H         SYMBOL        FONT16PX_240
  C:1CF9H         SYMBOL        FONT16PX_241
  C:1D0AH         SYMBOL        FONT16PX_242
  C:1D1BH         SYMBOL        FONT16PX_243
  C:1D2CH         SYMBOL        FONT16PX_244
  C:1D3DH         SYMBOL        FONT16PX_245
  C:1D4EH         SYMBOL        FONT16PX_246
  C:1D5FH         SYMBOL        FONT16PX_248
  C:1D70H         SYMBOL        FONT16PX_249
  C:1D81H         SYMBOL        FONT16PX_250
  C:1D92H         SYMBOL        FONT16PX_251
  C:1DA3H         SYMBOL        FONT16PX_252
  C:1DB4H         SYMBOL        FONT16PX_253
  C:1DC5H         SYMBOL        FONT16PX_254
  C:119EH         SYMBOL        FONT16PX_32
  C:11AFH         SYMBOL        FONT16PX_33
  C:11C0H         SYMBOL        FONT16PX_34
  C:11D1H         SYMBOL        FONT16PX_35
  C:11E2H         SYMBOL        FONT16PX_36
  C:11F3H         SYMBOL        FONT16PX_37
  C:1204H         SYMBOL        FONT16PX_38
  C:1215H         SYMBOL        FONT16PX_39
  C:1226H         SYMBOL        FONT16PX_40
BL51 BANKED LINKER/LOCATER V4.02                                                      05/28/2008  17:48:13  PAGE 31


  C:1237H         SYMBOL        FONT16PX_41
  C:1248H         SYMBOL        FONT16PX_42
  C:1259H         SYMBOL        FONT16PX_43
  C:126AH         SYMBOL        FONT16PX_44
  C:127BH         SYMBOL        FONT16PX_45
  C:128CH         SYMBOL        FONT16PX_46
  C:129DH         SYMBOL        FONT16PX_47
  C:12AEH         SYMBOL        FONT16PX_48
  C:12BFH         SYMBOL        FONT16PX_49
  C:12D0H         SYMBOL        FONT16PX_50
  C:12E1H         SYMBOL        FONT16PX_51
  C:12F2H         SYMBOL        FONT16PX_52
  C:1303H         SYMBOL        FONT16PX_53
  C:1314H         SYMBOL        FONT16PX_54
  C:1325H         SYMBOL        FONT16PX_55
  C:1336H         SYMBOL        FONT16PX_56
  C:1347H         SYMBOL        FONT16PX_57
  C:1358H         SYMBOL        FONT16PX_58
  C:1369H         SYMBOL        FONT16PX_59
  C:137AH         SYMBOL        FONT16PX_60
  C:138BH         SYMBOL        FONT16PX_61
  C:139CH         SYMBOL        FONT16PX_62
  C:13ADH         SYMBOL        FONT16PX_63
  C:13BEH         SYMBOL        FONT16PX_64
  C:13CFH         SYMBOL        FONT16PX_65
  C:13E0H         SYMBOL        FONT16PX_66
  C:13F1H         SYMBOL        FONT16PX_67
  C:1402H         SYMBOL        FONT16PX_68
  C:1413H         SYMBOL        FONT16PX_69
  C:1424H         SYMBOL        FONT16PX_70
  C:1435H         SYMBOL        FONT16PX_71
  C:1446H         SYMBOL        FONT16PX_72
  C:1457H         SYMBOL        FONT16PX_73
  C:1468H         SYMBOL        FONT16PX_74
  C:1479H         SYMBOL        FONT16PX_75
  C:148AH         SYMBOL        FONT16PX_76
  C:149BH         SYMBOL        FONT16PX_77
  C:14ACH         SYMBOL        FONT16PX_78
  C:14BDH         SYMBOL        FONT16PX_79
  C:14CEH         SYMBOL        FONT16PX_80
  C:14DFH         SYMBOL        FONT16PX_81
  C:14F0H         SYMBOL        FONT16PX_82
  C:1501H         SYMBOL        FONT16PX_83
  C:1512H         SYMBOL        FONT16PX_84
  C:1523H         SYMBOL        FONT16PX_85
  C:1534H         SYMBOL        FONT16PX_86
  C:1545H         SYMBOL        FONT16PX_87
  C:1556H         SYMBOL        FONT16PX_88
  C:1567H         SYMBOL        FONT16PX_89
  C:1578H         SYMBOL        FONT16PX_90
  C:1589H         SYMBOL        FONT16PX_91
  C:159AH         SYMBOL        FONT16PX_92
  C:15ABH         SYMBOL        FONT16PX_93
  C:15BCH         SYMBOL        FONT16PX_94
  C:15CDH         SYMBOL        FONT16PX_95
  C:15DEH         SYMBOL        FONT16PX_96
  C:15EFH         SYMBOL        FONT16PX_97
BL51 BANKED LINKER/LOCATER V4.02                                                      05/28/2008  17:48:13  PAGE 32


  C:1600H         SYMBOL        FONT16PX_98
  C:1611H         SYMBOL        FONT16PX_99
  C:1DD6H         SYMBOL        FONT16PX_BLANK
  N:0000H         SYMBOL        FONTS
  -------         ENDMOD        FONTS

  -------         MODULE        BUTTONS
  C:0000H         SYMBOL        _ICE_DUMMY_
  B:00D8H.2       PUBLIC        CCF2
  X:1506H         PUBLIC        btnact
  B:00D8H.3       PUBLIC        CCF3
  B:00D8H.4       PUBLIC        CCF4
  B:00D0H.6       PUBLIC        AC
  B:00B0H.4       PUBLIC        T0
  B:00B0H.5       PUBLIC        T1
  B:00A8H.7       PUBLIC        EA
  B:00A8H.6       PUBLIC        EC
  B:00D8H.7       PUBLIC        CF
  C:5903H         PUBLIC        ButtonsInit
  B:0098H.7       PUBLIC        FE
  B:00E8H.1       PUBLIC        EADC
  B:0080H.0       PUBLIC        P0_0
  B:0090H.0       PUBLIC        P1_0
  B:0080H.1       PUBLIC        P0_1
  D:003AH         PUBLIC        ebtnup
  B:00A0H.0       PUBLIC        P2_0
  B:0090H.1       PUBLIC        P1_1
  B:0080H.2       PUBLIC        P0_2
  B:00B0H.0       PUBLIC        P3_0
  B:00A0H.1       PUBLIC        P2_1
  B:0090H.2       PUBLIC        P1_2
  B:0080H.3       PUBLIC        P0_3
  B:00C0H.0       PUBLIC        P4_0
  B:00B0H.1       PUBLIC        P3_1
  B:00A0H.2       PUBLIC        P2_2
  B:0090H.3       PUBLIC        P1_3
  B:0080H.4       PUBLIC        P0_4
  B:00D8H.6       PUBLIC        CR
  B:00C0H.1       PUBLIC        P4_1
  B:00B0H.2       PUBLIC        P3_2
  B:00A0H.3       PUBLIC        P2_3
  B:0090H.4       PUBLIC        P1_4
  B:0080H.5       PUBLIC        P0_5
  B:00C8H.6       PUBLIC        EXF2
  B:00B0H.7       PUBLIC        RD
  B:00B0H.3       PUBLIC        P3_3
  B:00A0H.4       PUBLIC        P2_4
  B:0090H.5       PUBLIC        P1_5
  B:0080H.6       PUBLIC        P0_6
  B:00B0H.4       PUBLIC        P3_4
  B:00A0H.5       PUBLIC        P2_5
  B:0090H.6       PUBLIC        P1_6
  B:0080H.7       PUBLIC        P0_7
  B:00E8H.0       PUBLIC        ECAN
  B:00A8H.4       PUBLIC        ES
  B:00B0H.5       PUBLIC        P3_5
  B:00A0H.6       PUBLIC        P2_6
BL51 BANKED LINKER/LOCATER V4.02                                                      05/28/2008  17:48:13  PAGE 33


  B:0090H.7       PUBLIC        P1_7
  B:00D0H.1       PUBLIC        UD
  B:00B0H.6       PUBLIC        P3_6
  B:00A0H.7       PUBLIC        P2_7
  B:00B0H.7       PUBLIC        P3_7
  B:0098H.0       PUBLIC        RI
  B:00D0H.7       PUBLIC        CY
  B:00B0H.2       PUBLIC        INT0
  B:0098H.1       PUBLIC        TI
  B:00B0H.3       PUBLIC        INT1
  B:00D0H.2       PUBLIC        OV
  B:00C8H.1       PUBLIC        C_T2
  B:00B0H.6       PUBLIC        WR
  B:00C8H.5       PUBLIC        RCLK
  X:1556H         PUBLIC        last_scrN
  B:00C8H.4       PUBLIC        TCLK
  B:00E8H.2       PUBLIC        ETIM
  B:00E8H.3       PUBLIC        ESPI
  D:0089H         PUBLIC        TMOD
  B:0088H.1       PUBLIC        IE0
  B:0088H.3       PUBLIC        IE1
  C:5927H         PUBLIC        ClearActions
  X:1557H         PUBLIC        _last_scr
  C:5534H         PUBLIC        INTtimer0
  X:16D7H         PUBLIC        _this_scr
  B:00C8H.0       PUBLIC        CP_RL2
  B:00A8H.1       PUBLIC        ET0
  B:00A8H.3       PUBLIC        ET1
  B:0088H.5       PUBLIC        TF0
  B:00A8H.5       PUBLIC        ET2
  B:0088H.7       PUBLIC        TF1
  C:5192H         PUBLIC        _AddAction
  B:0098H.2       PUBLIC        RB8
  D:008CH         PUBLIC        TH0
  B:00C8H.7       PUBLIC        TF2
  B:00A8H.0       PUBLIC        EX0
  B:0088H.0       PUBLIC        IT0
  B:00A8H.2       PUBLIC        EX1
  B:0098H.3       PUBLIC        TB8
  B:0088H.2       PUBLIC        IT1
  B:00D0H.0       PUBLIC        P
  B:0098H.7       PUBLIC        SM0
  D:008AH         PUBLIC        TL0
  B:0098H.6       PUBLIC        SM1
  B:0098H.5       PUBLIC        SM2
  B:00D0H.3       PUBLIC        RS0
  B:0088H.4       PUBLIC        TR0
  B:00D0H.4       PUBLIC        RS1
  B:0088H.6       PUBLIC        TR1
  B:00C8H.2       PUBLIC        TR2
  D:003BH         PUBLIC        btn_last
  B:00C8H.3       PUBLIC        EXEN2
  C:4708H         PUBLIC        GUI
  B:0098H.4       PUBLIC        REN
  D:003CH         PUBLIC        ebtndown
  D:003DH         PUBLIC        btn_div
  B:00B0H.0       PUBLIC        RXD
BL51 BANKED LINKER/LOCATER V4.02                                                      05/28/2008  17:48:13  PAGE 34


  B:00B0H.1       PUBLIC        TXD
  B:00D0H.5       PUBLIC        F0
  B:00D8H.0       PUBLIC        CCF0
  B:00D8H.1       PUBLIC        CCF1
  -------         PROC          COM0021
  -------         ENDPROC       COM0021
  -------         PROC          CLEARACTIONS
  C:5927H         LINE#         29
  C:5927H         LINE#         30
  C:5927H         LINE#         31
  -------         ENDPROC       CLEARACTIONS
  -------         PROC          _ADDACTION
  D:0007H         SYMBOL        btn
  X:172DH         SYMBOL        type
  X:172EH         SYMBOL        gp
  X:1731H         SYMBOL        p1
  X:1733H         SYMBOL        p2
  X:1735H         SYMBOL        p3
  -------         DO            p3
  C:000EH         SYMBOL        btnmap
  X:1737H         SYMBOL        abp
  -------         ENDDO         abp
  C:5192H         LINE#         37
  C:519CH         LINE#         40
  C:51C9H         LINE#         42
  C:51D8H         LINE#         43
  C:51F0H         LINE#         44
  C:5207H         LINE#         45
  C:5217H         LINE#         46
  -------         ENDPROC       _ADDACTION
  -------         PROC          BUTTONSINIT
  C:5903H         LINE#         52
  C:5903H         LINE#         53
  C:5903H         LINE#         55
  C:5909H         LINE#         56
  C:590CH         LINE#         57
  C:590EH         LINE#         58
  C:5910H         LINE#         60
  C:5913H         LINE#         62
  C:5915H         LINE#         63
  C:5917H         LINE#         64
  -------         ENDPROC       BUTTONSINIT
  -------         PROC          INTTIMER0
  -------         DO            INTTIMER0
  D:001FH         SYMBOL        btn_state
  D:001EH         SYMBOL        btn_up
  D:001DH         SYMBOL        btn_down
  -------         ENDDO         btn_down
  C:5534H         LINE#         69
  C:553FH         LINE#         74
  C:5541H         LINE#         77
  C:5543H         LINE#         78
  C:5549H         LINE#         79
  C:554BH         LINE#         82
  C:5551H         LINE#         83
  C:5551H         LINE#         84
  C:5554H         LINE#         87
BL51 BANKED LINKER/LOCATER V4.02                                                      05/28/2008  17:48:13  PAGE 35


  C:555AH         LINE#         88
  C:555FH         LINE#         89
  C:5563H         LINE#         90
  C:5565H         LINE#         92
  C:556AH         LINE#         97
  C:5584H         LINE#         98
  C:5587H         LINE#         100
  C:558AH         LINE#         101
  C:558DH         LINE#         102
  C:558DH         LINE#         103
  -------         ENDPROC       INTTIMER0
  -------         PROC          GUI
  -------         DO            GUI
  D:0022H         SYMBOL        i
  X:172CH         SYMBOL        paint
  X:172DH         SYMBOL        gp
  X:1730H         SYMBOL        p1
  X:1732H         SYMBOL        p2
  X:1734H         SYMBOL        p3
  -------         ENDDO         p3
  C:4708H         LINE#         109
  C:4708H         LINE#         110
  C:4708H         LINE#         112
  C:470DH         LINE#         117
  C:470FH         LINE#         118
  C:470FH         LINE#         119
  C:4723H         LINE#         120
  C:4723H         LINE#         122
  C:473CH         LINE#         123
  C:474CH         LINE#         124
  C:475CH         LINE#         125
  C:476CH         LINE#         128
  C:4793H         LINE#         129
  C:4793H         LINE#         131
  C:4793H         LINE#         132
  C:47ABH         LINE#         133
  C:47B1H         LINE#         134
  C:47B4H         LINE#         135
  C:47B7H         LINE#         136
  C:47BAH         LINE#         138
  C:47BAH         LINE#         139
  C:47C3H         LINE#         140
  C:47C3H         LINE#         141
  C:47CFH         LINE#         142
  C:47D2H         LINE#         143
  C:47D2H         LINE#         144
  C:47D5H         LINE#         145
  C:47D8H         LINE#         147
  C:47D8H         LINE#         148
  C:47E2H         LINE#         149
  C:480AH         LINE#         150
  C:482DH         LINE#         151
  C:4830H         LINE#         152
  C:4833H         LINE#         154
  C:4833H         LINE#         155
  C:4842H         LINE#         156
  C:485DH         LINE#         157
BL51 BANKED LINKER/LOCATER V4.02                                                      05/28/2008  17:48:13  PAGE 36


  C:4878H         LINE#         158
  C:487BH         LINE#         159
  C:487DH         LINE#         161
  C:487DH         LINE#         162
  C:4887H         LINE#         163
  C:488AH         LINE#         164
  C:488AH         LINE#         165
  C:488AH         LINE#         166
  C:488DH         LINE#         167
  C:488DH         LINE#         168
  C:4899H         LINE#         172
  C:48A3H         LINE#         173
  C:48A3H         LINE#         174
  C:48B2H         LINE#         175
  C:48D3H         LINE#         176
  C:48D6H         LINE#         177
  C:48D9H         LINE#         178
  C:48D9H         LINE#         179
  -------         ENDPROC       GUI
  -------         ENDMOD        BUTTONS

  -------         MODULE        MODBUS
  C:0000H         SYMBOL        _ICE_DUMMY_
  B:00D8H.2       PUBLIC        CCF2
  B:00D8H.3       PUBLIC        CCF3
  B:00D8H.4       PUBLIC        CCF4
  C:5849H         PUBLIC        MODBUSinit
  B:00D0H.6       PUBLIC        AC
  B:00B0H.4       PUBLIC        T0
  B:00B0H.5       PUBLIC        T1
  X:1300H         PUBLIC        COMbuffRxPos
  B:00A8H.7       PUBLIC        EA
  X:1302H         PUBLIC        MODBUScomEvents
  X:1304H         PUBLIC        COMbuffTxPos
  B:00A8H.6       PUBLIC        EC
  B:00D8H.7       PUBLIC        CF
  C:544DH         PUBLIC        INT_UART
  B:0098H.7       PUBLIC        FE
  B:00E8H.1       PUBLIC        EADC
  B:0080H.0       PUBLIC        P0_0
  B:0090H.0       PUBLIC        P1_0
  B:0080H.1       PUBLIC        P0_1
  D:00B7H         PUBLIC        IPH0
  B:00A0H.0       PUBLIC        P2_0
  B:0090H.1       PUBLIC        P1_1
  B:0080H.2       PUBLIC        P0_2
  B:00B0H.0       PUBLIC        P3_0
  B:00A0H.1       PUBLIC        P2_1
  B:0090H.2       PUBLIC        P1_2
  B:0080H.3       PUBLIC        P0_3
  B:00C0H.0       PUBLIC        P4_0
  B:00B0H.1       PUBLIC        P3_1
  B:00A0H.2       PUBLIC        P2_2
  B:0090H.3       PUBLIC        P1_3
  B:0080H.4       PUBLIC        P0_4
  B:00D8H.6       PUBLIC        CR
  B:00C0H.1       PUBLIC        P4_1
BL51 BANKED LINKER/LOCATER V4.02                                                      05/28/2008  17:48:13  PAGE 37


  B:00B0H.2       PUBLIC        P3_2
  B:00A0H.3       PUBLIC        P2_3
  B:0090H.4       PUBLIC        P1_4
  B:0080H.5       PUBLIC        P0_5
  D:00B8H         PUBLIC        IPL0
  B:00C8H.6       PUBLIC        EXF2
  B:00B0H.7       PUBLIC        RD
  B:00B0H.3       PUBLIC        P3_3
  B:00A0H.4       PUBLIC        P2_4
  B:0090H.5       PUBLIC        P1_5
  B:0080H.6       PUBLIC        P0_6
  B:00B0H.4       PUBLIC        P3_4
  B:00A0H.5       PUBLIC        P2_5
  B:0090H.6       PUBLIC        P1_6
  B:0080H.7       PUBLIC        P0_7
  B:00E8H.0       PUBLIC        ECAN
  B:00A8H.4       PUBLIC        ES
  B:00B0H.5       PUBLIC        P3_5
  B:00A0H.6       PUBLIC        P2_6
  B:0090H.7       PUBLIC        P1_7
  B:00D0H.1       PUBLIC        UD
  B:00B0H.6       PUBLIC        P3_6
  B:00A0H.7       PUBLIC        P2_7
  B:00B0H.7       PUBLIC        P3_7
  B:0098H.0       PUBLIC        RI
  B:00D0H.7       PUBLIC        CY
  B:00B0H.2       PUBLIC        INT0
  B:0098H.1       PUBLIC        TI
  B:00B0H.3       PUBLIC        INT1
  C:5936H         PUBLIC        INT_timer1
  D:00CBH         PUBLIC        RCAP2H
  B:00D0H.2       PUBLIC        OV
  D:00CAH         PUBLIC        RCAP2L
  B:00C8H.1       PUBLIC        C_T2
  B:00B0H.6       PUBLIC        WR
  B:00C8H.5       PUBLIC        RCLK
  B:00C8H.4       PUBLIC        TCLK
  B:00E8H.2       PUBLIC        ETIM
  X:1305H         PUBLIC        COMbuffRX
  D:0099H         PUBLIC        SBUF
  B:00E8H.3       PUBLIC        ESPI
  X:1405H         PUBLIC        COMbuffTX
  D:0098H         PUBLIC        SCON
  D:0089H         PUBLIC        TMOD
  D:0042H         PUBLIC        MODBUS_timeout
  B:0088H.1       PUBLIC        IE0
  B:0088H.3       PUBLIC        IE1
  B:00C8H.0       PUBLIC        CP_RL2
  B:00A8H.1       PUBLIC        ET0
  B:00A8H.3       PUBLIC        ET1
  B:0088H.5       PUBLIC        TF0
  B:00A8H.5       PUBLIC        ET2
  B:0088H.7       PUBLIC        TF1
  C:391AH         PUBLIC        MODBUS
  B:0098H.2       PUBLIC        RB8
  B:00C8H.7       PUBLIC        TF2
  B:00A8H.0       PUBLIC        EX0
BL51 BANKED LINKER/LOCATER V4.02                                                      05/28/2008  17:48:13  PAGE 38


  D:008DH         PUBLIC        TH1
  B:0088H.0       PUBLIC        IT0
  B:00A8H.2       PUBLIC        EX1
  B:0098H.3       PUBLIC        TB8
  D:00CDH         PUBLIC        TH2
  B:0088H.2       PUBLIC        IT1
  B:00D0H.0       PUBLIC        P
  B:0098H.7       PUBLIC        SM0
  B:0098H.6       PUBLIC        SM1
  D:008BH         PUBLIC        TL1
  B:0098H.5       PUBLIC        SM2
  D:00CCH         PUBLIC        TL2
  B:00D0H.3       PUBLIC        RS0
  B:0088H.4       PUBLIC        TR0
  B:00D0H.4       PUBLIC        RS1
  B:0088H.6       PUBLIC        TR1
  B:00C8H.2       PUBLIC        TR2
  B:00C8H.3       PUBLIC        EXEN2
  B:0098H.4       PUBLIC        REN
  D:00C8H         PUBLIC        T2CON
  B:00B0H.0       PUBLIC        RXD
  B:00B0H.1       PUBLIC        TXD
  X:1505H         PUBLIC        COMbuffTxLen
  B:00D0H.5       PUBLIC        F0
  B:00D8H.0       PUBLIC        CCF0
  B:00D8H.1       PUBLIC        CCF1
  -------         PROC          COM0040
  -------         ENDPROC       COM0040
  -------         PROC          MODBUSINIT
  C:5849H         LINE#         23
  C:5849H         LINE#         24
  C:5849H         LINE#         26
  C:584CH         LINE#         27
  C:584FH         LINE#         28
  C:5855H         LINE#         29
  C:585BH         LINE#         30
  C:585DH         LINE#         31
  C:585FH         LINE#         33
  C:5868H         LINE#         34
  C:586BH         LINE#         37
  C:586DH         LINE#         40
  C:5870H         LINE#         41
  C:5873H         LINE#         42
  C:5875H         LINE#         43
  C:5877H         LINE#         45
  C:5879H         LINE#         48
  C:587CH         LINE#         49
  C:587FH         LINE#         52
  C:5883H         LINE#         53
  -------         ENDPROC       MODBUSINIT
  -------         PROC          INT_TIMER1
  C:5936H         LINE#         58
  C:5936H         LINE#         60
  C:5938H         LINE#         61
  C:593BH         LINE#         62
  C:593DH         LINE#         63
  C:593FH         LINE#         66
BL51 BANKED LINKER/LOCATER V4.02                                                      05/28/2008  17:48:13  PAGE 39


  C:593FH         LINE#         67
  C:5942H         LINE#         68
  C:5944H         LINE#         69
  C:5944H         LINE#         70
  -------         ENDPROC       INT_TIMER1
  -------         PROC          INT_UART
  C:544DH         LINE#         75
  C:545AH         LINE#         77
  C:545DH         LINE#         78
  C:545DH         LINE#         82
  C:546AH         LINE#         83
  C:546AH         LINE#         85
  C:546CH         LINE#         86
  C:547DH         LINE#         87
  C:547FH         LINE#         89
  C:547FH         LINE#         91
  C:5481H         LINE#         92
  C:5486H         LINE#         93
  C:5486H         LINE#         95
  C:5488H         LINE#         96
  C:5488H         LINE#         98
  C:548BH         LINE#         99
  C:548BH         LINE#         103
  C:5494H         LINE#         104
  C:5494H         LINE#         105
  C:54AAH         LINE#         108
  C:54ADH         LINE#         109
  C:54AFH         LINE#         110
  C:54B2H         LINE#         111
  C:54B4H         LINE#         112
  C:54B4H         LINE#         114
  C:54B6H         LINE#         115
  C:54B6H         LINE#         116
  -------         ENDPROC       INT_UART
  -------         PROC          MODBUS
  -------         DO            MODBUS
  X:172CH         SYMBOL        rdaddr
  X:172EH         SYMBOL        wraddr
  X:1730H         SYMBOL        rdlen
  X:1731H         SYMBOL        wrlen
  X:1732H         SYMBOL        dptr
  C:3C74H         SYMBOL        unknownf
  -------         ENDDO         unknownf
  C:391AH         LINE#         121
  C:391AH         LINE#         122
  C:391AH         LINE#         127
  C:391CH         LINE#         128
  C:3925H         LINE#         129
  C:3925H         LINE#         130
  C:3942H         LINE#         131
  C:3942H         LINE#         132
  C:396EH         LINE#         133
  C:396EH         LINE#         134
  C:398AH         LINE#         135
  C:398AH         LINE#         136
  C:398AH         LINE#         140
  C:398DH         LINE#         141
BL51 BANKED LINKER/LOCATER V4.02                                                      05/28/2008  17:48:13  PAGE 40


  C:398DH         LINE#         142
  C:3992H         LINE#         143
  C:3997H         LINE#         144
  C:399FH         LINE#         145
  C:39B2H         LINE#         148
  C:39B8H         LINE#         149
  C:39B8H         LINE#         150
  C:39B8H         LINE#         151
  C:39C0H         LINE#         152
  C:39C3H         LINE#         153
  C:39C3H         LINE#         157
  C:39CEH         LINE#         158
  C:39CEH         LINE#         159
  C:39CEH         LINE#         160
  C:39CEH         LINE#         161
  C:39D3H         LINE#         162
  C:39D9H         LINE#         163
  C:39E2H         LINE#         164
  C:39E7H         LINE#         165
  C:39ECH         LINE#         166
  C:39F4H         LINE#         167
  C:39FDH         LINE#         168
  C:3A07H         LINE#         171
  C:3A1AH         LINE#         172
  C:3A1AH         LINE#         173
  C:3A1AH         LINE#         174
  C:3A1FH         LINE#         175
  C:3A2CH         LINE#         176
  C:3A34H         LINE#         177
  C:3A37H         LINE#         178
  C:3A37H         LINE#         179
  C:3A3CH         LINE#         180
  C:3A49H         LINE#         181
  C:3A51H         LINE#         182
  C:3A54H         LINE#         183
  C:3A54H         LINE#         184
  C:3A59H         LINE#         185
  C:3A66H         LINE#         186
  C:3A6EH         LINE#         187
  C:3A71H         LINE#         188
  C:3A71H         LINE#         189
  C:3A76H         LINE#         190
  C:3A83H         LINE#         191
  C:3A8BH         LINE#         192
  C:3A8DH         LINE#         193
  C:3A8DH         LINE#         194
  C:3A92H         LINE#         195
  C:3A9FH         LINE#         196
  C:3AA7H         LINE#         197
  C:3AA9H         LINE#         198
  C:3AA9H         LINE#         200
  C:3AA9H         LINE#         201
  C:3AA9H         LINE#         202
  C:3AA9H         LINE#         203
  C:3AA9H         LINE#         204
  C:3AACH         LINE#         205
  C:3AACH         LINE#         206
BL51 BANKED LINKER/LOCATER V4.02                                                      05/28/2008  17:48:13  PAGE 41


  C:3AACH         LINE#         208
  C:3AB2H         LINE#         209
  C:3AB2H         LINE#         210
  C:3AB2H         LINE#         211
  C:3ABAH         LINE#         212
  C:3ABDH         LINE#         214
  C:3ABDH         LINE#         215
  C:3ABDH         LINE#         216
  C:3ABDH         LINE#         222
  C:3ACCH         LINE#         223
  C:3AD4H         LINE#         225
  C:3AE4H         LINE#         226
  C:3AECH         LINE#         231
  C:3AF5H         LINE#         232
  C:3AF5H         LINE#         233
  C:3B02H         LINE#         234
  C:3B0BH         LINE#         235
  C:3B14H         LINE#         236
  C:3B1DH         LINE#         237
  C:3B29H         LINE#         238
  C:3B29H         LINE#         241
  C:3B3DH         LINE#         242
  C:3B49H         LINE#         245
  C:3B58H         LINE#         246
  C:3B58H         LINE#         247
  C:3B5EH         LINE#         248
  C:3B62H         LINE#         249
  C:3B62H         LINE#         252
  C:3B65H         LINE#         253
  C:3B6BH         LINE#         254
  C:3B75H         LINE#         260
  C:3B87H         LINE#         261
  C:3B87H         LINE#         262
  C:3B90H         LINE#         263
  C:3BCEH         LINE#         264
  C:3BCEH         LINE#         267
  C:3BD4H         LINE#         268
  C:3BD4H         LINE#         269
  C:3BD4H         LINE#         270
  C:3BDCH         LINE#         272
  C:3BDFH         LINE#         273
  C:3BDFH         LINE#         277
  C:3BE9H         LINE#         278
  C:3BE9H         LINE#         279
  C:3BE9H         LINE#         281
  C:3BE9H         LINE#         282
  C:3BE9H         LINE#         283
  C:3BF1H         LINE#         284
  C:3BF1H         LINE#         285
  C:3BF1H         LINE#         286
  C:3BF6H         LINE#         287
  C:3BFAH         LINE#         288
  C:3C00H         LINE#         289
  C:3C08H         LINE#         290
  C:3C1FH         LINE#         291
  C:3C22H         LINE#         292
  C:3C25H         LINE#         293
BL51 BANKED LINKER/LOCATER V4.02                                                      05/28/2008  17:48:13  PAGE 42


  C:3C25H         LINE#         295
  C:3C25H         LINE#         296
  C:3C25H         LINE#         297
  C:3C2DH         LINE#         298
  C:3C2DH         LINE#         299
  C:3C2DH         LINE#         300
  C:3C32H         LINE#         301
  C:3C37H         LINE#         302
  C:3C3DH         LINE#         303
  C:3C45H         LINE#         304
  C:3C5CH         LINE#         305
  C:3C5FH         LINE#         306
  C:3C61H         LINE#         307
  C:3C61H         LINE#         309
  C:3C61H         LINE#         310
  C:3C61H         LINE#         311
  C:3C61H         LINE#         312
  C:3C61H         LINE#         313
  C:3C64H         LINE#         314
  C:3C64H         LINE#         315
  C:3C64H         LINE#         318
  C:3C6AH         LINE#         319
  C:3C6AH         LINE#         320
  C:3C6AH         LINE#         321
  C:3C72H         LINE#         322
  C:3C74H         LINE#         323
  C:3C74H         LINE#         324
  C:3C74H         LINE#         326
  C:3C7AH         LINE#         327
  C:3C84H         LINE#         328
  C:3C88H         LINE#         329
  C:3C99H         LINE#         330
  C:3C9FH         LINE#         331
  C:3CA1H         LINE#         332
  C:3CA1H         LINE#         333
  C:3CA1H         LINE#         334
  C:3CA1H         LINE#         335
  C:3CA4H         LINE#         336
  C:3CA6H         LINE#         338
  C:3CA9H         LINE#         339
  C:3CA9H         LINE#         340
  C:3CABH         LINE#         341
  -------         ENDPROC       MODBUS
  -------         ENDMOD        MODBUS

  -------         MODULE        MODBUS_ROUTINES
  C:44E4H         SEGMENT       ?PR?_CRC16?MODBUS_ROUTINES
  C:44E4H         PUBLIC        _CRC16
  D:00A2H         SYMBOL        AUXR1
  C:44F1H         SYMBOL        CRC16L1
  C:4508H         SYMBOL        CRC16_DATAH
  C:4608H         SYMBOL        CRC16_DATAL
  D:0083H         SYMBOL        DPH
  D:0082H         SYMBOL        DPL
  N:0000H         SYMBOL        MODBUS_ROUTINES
  C:44E4H         LINE#         17
  C:44E7H         LINE#         18
BL51 BANKED LINKER/LOCATER V4.02                                                      05/28/2008  17:48:13  PAGE 43


  C:44E9H         LINE#         19
  C:44EBH         LINE#         20
  C:44EDH         LINE#         21
  C:44EFH         LINE#         22
  C:44F1H         LINE#         23
  C:44F2H         LINE#         24
  C:44F3H         LINE#         25
  C:44F5H         LINE#         26
  C:44F6H         LINE#         27
  C:44F7H         LINE#         28
  C:44F8H         LINE#         29
  C:44F9H         LINE#         30
  C:44FAH         LINE#         31
  C:44FDH         LINE#         32
  C:44FEH         LINE#         33
  C:44FFH         LINE#         34
  C:4500H         LINE#         35
  C:4503H         LINE#         36
  C:4505H         LINE#         37
  C:4507H         LINE#         38
  -------         ENDMOD        MODBUS_ROUTINES

  -------         MODULE        E3D_DEMO
  C:0000H         SYMBOL        _ICE_DUMMY_
  C:354EH         PUBLIC        sinT
  C:55F7H         PUBLIC        _E3D_demo
  X:16DAH         PUBLIC        E3D_points
  C:38D2H         PUBLIC        obj1_vertexT
  C:3902H         PUBLIC        obj2_vertexT
  C:38EAH         PUBLIC        obj1_wireT
  C:390EH         PUBLIC        obj2_wireT
  C:54C1H         PUBLIC        _E3D_DrawObject
  C:4297H         PUBLIC        _E3D_make_move_rotate_transform
  C:52B9H         PUBLIC        _E3D_Rotate
  X:16EAH         PUBLIC        E3Dobj
  C:4038H         PUBLIC        _E3D_RandomMove
  -------         PROC          COM0023
  -------         ENDPROC       COM0023
  -------         PROC          _E3D_MAKE_MOVE_ROTATE_TRANSFORM
  D:0007H         SYMBOL        objid
  -------         DO            objid
  X:172CH         SYMBOL        i
  D:0006H         SYMBOL        obj
  X:172DH         SYMBOL        vp
  X:172FH         SYMBOL        vnum
  X:1730H         SYMBOL        x
  X:1732H         SYMBOL        y
  X:1734H         SYMBOL        z
  X:1736H         SYMBOL        tmp
  X:1738H         SYMBOL        xpos
  X:1739H         SYMBOL        ypos
  X:173AH         SYMBOL        zpos
  X:173CH         SYMBOL        xrot
  X:173EH         SYMBOL        yrot
  -------         ENDDO         yrot
  C:4297H         LINE#         84
  C:4297H         LINE#         87
BL51 BANKED LINKER/LOCATER V4.02                                                      05/28/2008  17:48:13  PAGE 44


  C:429BH         LINE#         88
  C:42A4H         LINE#         89
  C:42AFH         LINE#         91
  C:42BAH         LINE#         92
  C:42C5H         LINE#         93
  C:42D3H         LINE#         94
  C:42E1H         LINE#         95
  C:42F4H         LINE#         98
  C:4309H         LINE#         99
  C:4309H         LINE#         101
  C:4310H         LINE#         102
  C:4316H         LINE#         103
  C:4320H         LINE#         106
  C:4352H         LINE#         107
  C:4383H         LINE#         108
  C:438EH         LINE#         111
  C:43D5H         LINE#         112
  C:4429H         LINE#         113
  C:4438H         LINE#         116
  C:444AH         LINE#         117
  C:445CH         LINE#         118
  C:4476H         LINE#         121
  C:44A8H         LINE#         122
  C:44DAH         LINE#         123
  C:44E3H         LINE#         124
  -------         ENDPROC       _E3D_MAKE_MOVE_ROTATE_TRANSFORM
  -------         PROC          _E3D_DRAWOBJECT
  D:0007H         SYMBOL        objid
  -------         DO            objid
  X:172CH         SYMBOL        i
  D:0006H         SYMBOL        obj
  X:172DH         SYMBOL        wp
  X:172FH         SYMBOL        wnum
  -------         ENDDO         wnum
  C:54C1H         LINE#         130
  C:54C1H         LINE#         133
  C:54C5H         LINE#         134
  C:54D0H         LINE#         135
  C:54DCH         LINE#         137
  C:54EEH         LINE#         138
  C:54EEH         LINE#         139
  C:552AH         LINE#         140
  C:5533H         LINE#         141
  -------         ENDPROC       _E3D_DRAWOBJECT
  -------         PROC          _E3D_ROTATE
  D:0007H         SYMBOL        objid
  X:172CH         SYMBOL        xrot
  D:0001H         SYMBOL        yrot
  -------         DO            yrot
  X:172DH         SYMBOL        obj
  D:0004H         SYMBOL        E3D_xrot
  D:0006H         SYMBOL        E3D_yrot
  -------         ENDDO         E3D_yrot
  C:52B9H         LINE#         147
  C:52C0H         LINE#         149
  C:52CAH         LINE#         150
  C:52DBH         LINE#         151
BL51 BANKED LINKER/LOCATER V4.02                                                      05/28/2008  17:48:13  PAGE 45


  C:52E5H         LINE#         154
  C:52F4H         LINE#         155
  C:5307H         LINE#         156
  C:5314H         LINE#         157
  C:5327H         LINE#         159
  C:533CH         LINE#         160
  -------         ENDPROC       _E3D_ROTATE
  -------         PROC          _E3D_RANDOMMOVE
  D:0007H         SYMBOL        objid
  -------         DO            objid
  X:172CH         SYMBOL        obj
  X:172EH         SYMBOL        E3D_xposdest
  X:172FH         SYMBOL        E3D_yposdest
  X:1730H         SYMBOL        E3D_zposdest
  X:1731H         SYMBOL        E3D_xspd
  X:1733H         SYMBOL        E3D_yspd
  X:1735H         SYMBOL        E3D_zspd
  X:1737H         SYMBOL        E3D_xpos
  X:1738H         SYMBOL        E3D_ypos
  X:1739H         SYMBOL        E3D_zpos
  -------         ENDDO         E3D_zpos
  C:4038H         LINE#         167
  C:4038H         LINE#         169
  C:4042H         LINE#         170
  C:4054H         LINE#         171
  C:405EH         LINE#         172
  C:4068H         LINE#         173
  C:407EH         LINE#         174
  C:408FH         LINE#         175
  C:40A0H         LINE#         176
  C:40B1H         LINE#         177
  C:40BBH         LINE#         178
  C:40CCH         LINE#         181
  C:40D7H         LINE#         182
  C:40D7H         LINE#         183
  C:40EEH         LINE#         184
  C:40EEH         LINE#         185
  C:40F6H         LINE#         186
  C:40F9H         LINE#         187
  C:40FBH         LINE#         189
  C:40FBH         LINE#         190
  C:4118H         LINE#         191
  C:4118H         LINE#         192
  C:4123H         LINE#         193
  C:4126H         LINE#         194
  C:4126H         LINE#         197
  C:4133H         LINE#         198
  C:4133H         LINE#         199
  C:414AH         LINE#         200
  C:414DH         LINE#         201
  C:4152H         LINE#         202
  C:4155H         LINE#         203
  C:4157H         LINE#         205
  C:4157H         LINE#         206
  C:4174H         LINE#         207
  C:4177H         LINE#         208
  C:4187H         LINE#         209
BL51 BANKED LINKER/LOCATER V4.02                                                      05/28/2008  17:48:13  PAGE 46


  C:418AH         LINE#         210
  C:418AH         LINE#         213
  C:419CH         LINE#         214
  C:419CH         LINE#         215
  C:41B3H         LINE#         216
  C:41B6H         LINE#         217
  C:41BDH         LINE#         218
  C:41C0H         LINE#         219
  C:41C2H         LINE#         221
  C:41C2H         LINE#         222
  C:41DFH         LINE#         223
  C:41E2H         LINE#         224
  C:41F4H         LINE#         225
  C:41F7H         LINE#         226
  C:41F7H         LINE#         229
  C:4209H         LINE#         230
  C:4214H         LINE#         231
  C:421FH         LINE#         232
  C:422AH         LINE#         233
  C:4235H         LINE#         234
  C:4240H         LINE#         235
  C:424BH         LINE#         236
  C:4256H         LINE#         237
  C:4261H         LINE#         238
  -------         ENDPROC       _E3D_RANDOMMOVE
  -------         PROC          _E3D_DEMO
  D:0007H         SYMBOL        events
  C:55F7H         LINE#         245
  C:55F7H         LINE#         246
  C:55F7H         LINE#         247
  C:5605H         LINE#         250
  C:5608H         LINE#         251
  C:5608H         LINE#         252
  C:560BH         LINE#         253
  C:5627H         LINE#         254
  C:5627H         LINE#         257
  C:562CH         LINE#         258
  C:5631H         LINE#         259
  C:5636H         LINE#         260
  C:563BH         LINE#         263
  C:5644H         LINE#         264
  C:564DH         LINE#         266
  C:5652H         LINE#         267
  -------         ENDPROC       _E3D_DEMO
  -------         ENDMOD        E3D_DEMO

  -------         MODULE        SCREENS
  C:0000H         SYMBOL        _ICE_DUMMY_
  B:00D8H.2       PUBLIC        CCF2
  B:00D8H.3       PUBLIC        CCF3
  B:00D8H.4       PUBLIC        CCF4
  B:00D0H.6       PUBLIC        AC
  B:00B0H.4       PUBLIC        T0
  B:00B0H.5       PUBLIC        T1
  B:00A8H.7       PUBLIC        EA
  B:00A8H.6       PUBLIC        EC
  B:00D8H.7       PUBLIC        CF
BL51 BANKED LINKER/LOCATER V4.02                                                      05/28/2008  17:48:13  PAGE 47


  B:0098H.7       PUBLIC        FE
  B:00E8H.1       PUBLIC        EADC
  B:0080H.0       PUBLIC        P0_0
  B:0090H.0       PUBLIC        P1_0
  B:0080H.1       PUBLIC        P0_1
  B:00A0H.0       PUBLIC        P2_0
  B:0090H.1       PUBLIC        P1_1
  B:0080H.2       PUBLIC        P0_2
  B:00B0H.0       PUBLIC        P3_0
  B:00A0H.1       PUBLIC        P2_1
  B:0090H.2       PUBLIC        P1_2
  B:0080H.3       PUBLIC        P0_3
  B:00C0H.0       PUBLIC        P4_0
  B:00B0H.1       PUBLIC        P3_1
  B:00A0H.2       PUBLIC        P2_2
  B:0090H.3       PUBLIC        P1_3
  B:0080H.4       PUBLIC        P0_4
  B:00D8H.6       PUBLIC        CR
  B:00C0H.1       PUBLIC        P4_1
  B:00B0H.2       PUBLIC        P3_2
  B:00A0H.3       PUBLIC        P2_3
  B:0090H.4       PUBLIC        P1_4
  B:0080H.5       PUBLIC        P0_5
  B:00C8H.6       PUBLIC        EXF2
  B:00B0H.7       PUBLIC        RD
  B:00B0H.3       PUBLIC        P3_3
  B:00A0H.4       PUBLIC        P2_4
  B:0090H.5       PUBLIC        P1_5
  B:0080H.6       PUBLIC        P0_6
  B:00B0H.4       PUBLIC        P3_4
  B:00A0H.5       PUBLIC        P2_5
  B:0090H.6       PUBLIC        P1_6
  B:0080H.7       PUBLIC        P0_7
  B:00E8H.0       PUBLIC        ECAN
  B:00A8H.4       PUBLIC        ES
  B:00B0H.5       PUBLIC        P3_5
  B:00A0H.6       PUBLIC        P2_6
  B:0090H.7       PUBLIC        P1_7
  B:00D0H.1       PUBLIC        UD
  B:00B0H.6       PUBLIC        P3_6
  B:00A0H.7       PUBLIC        P2_7
  B:00B0H.7       PUBLIC        P3_7
  B:0098H.0       PUBLIC        RI
  B:00D0H.7       PUBLIC        CY
  B:00B0H.2       PUBLIC        INT0
  B:0098H.1       PUBLIC        TI
  B:00B0H.3       PUBLIC        INT1
  B:00D0H.2       PUBLIC        OV
  B:00C8H.1       PUBLIC        C_T2
  B:00B0H.6       PUBLIC        WR
  B:00C8H.5       PUBLIC        RCLK
  B:00C8H.4       PUBLIC        TCLK
  B:00E8H.2       PUBLIC        ETIM
  B:00E8H.3       PUBLIC        ESPI
  C:2962H         PUBLIC        icon_0
  C:2A64H         PUBLIC        icon_1
  B:0088H.1       PUBLIC        IE0
BL51 BANKED LINKER/LOCATER V4.02                                                      05/28/2008  17:48:13  PAGE 48


  B:0088H.3       PUBLIC        IE1
  B:00C8H.0       PUBLIC        CP_RL2
  B:00A8H.1       PUBLIC        ET0
  B:00A8H.3       PUBLIC        ET1
  B:0088H.5       PUBLIC        TF0
  B:00A8H.5       PUBLIC        ET2
  B:0088H.7       PUBLIC        TF1
  B:0098H.2       PUBLIC        RB8
  B:00C8H.7       PUBLIC        TF2
  B:00A8H.0       PUBLIC        EX0
  B:0088H.0       PUBLIC        IT0
  B:00A8H.2       PUBLIC        EX1
  B:0098H.3       PUBLIC        TB8
  B:0088H.2       PUBLIC        IT1
  B:00D0H.0       PUBLIC        P
  B:0098H.7       PUBLIC        SM0
  B:0098H.6       PUBLIC        SM1
  B:0098H.5       PUBLIC        SM2
  B:00D0H.3       PUBLIC        RS0
  B:0088H.4       PUBLIC        TR0
  B:00D0H.4       PUBLIC        RS1
  B:0088H.6       PUBLIC        TR1
  B:00C8H.2       PUBLIC        TR2
  B:00C8H.3       PUBLIC        EXEN2
  B:0098H.4       PUBLIC        REN
  B:00B0H.0       PUBLIC        RXD
  B:00B0H.1       PUBLIC        TXD
  C:50E8H         PUBLIC        _Screen1
  C:500DH         PUBLIC        _Screen2
  B:00D0H.5       PUBLIC        F0
  C:48DAH         PUBLIC        _Screen3
  B:00D8H.0       PUBLIC        CCF0
  B:00D8H.1       PUBLIC        CCF1
  -------         PROC          COM0009
  -------         ENDPROC       COM0009
  -------         PROC          _SCREEN1
  D:0007H         SYMBOL        events
  C:50E8H         LINE#         124
  C:50E8H         LINE#         125
  C:50E8H         LINE#         126
  C:50F2H         LINE#         129
  C:50F5H         LINE#         130
  C:50F5H         LINE#         131
  C:50F8H         LINE#         132
  C:510CH         LINE#         133
  C:510CH         LINE#         136
  C:511EH         LINE#         137
  C:512DH         LINE#         138
  C:513CH         LINE#         139
  C:514BH         LINE#         140
  C:515DH         LINE#         141
  C:516FH         LINE#         142
  C:517EH         LINE#         143
  -------         ENDPROC       _SCREEN1
  -------         PROC          _SCREEN2
  D:0007H         SYMBOL        events
  C:500DH         LINE#         149
BL51 BANKED LINKER/LOCATER V4.02                                                      05/28/2008  17:48:13  PAGE 49


  C:500DH         LINE#         150
  C:500DH         LINE#         151
  C:5017H         LINE#         154
  C:501CH         LINE#         155
  C:501CH         LINE#         156
  C:501FH         LINE#         157
  C:5033H         LINE#         158
  C:5047H         LINE#         159
  C:505BH         LINE#         160
  C:505BH         LINE#         163
  C:506CH         LINE#         164
  C:5081H         LINE#         165
  C:5096H         LINE#         166
  C:50A8H         LINE#         167
  C:50B7H         LINE#         168
  C:50C9H         LINE#         169
  C:50DEH         LINE#         170
  -------         ENDPROC       _SCREEN2
  -------         PROC          _SCREEN3
  D:0007H         SYMBOL        events
  C:48DAH         LINE#         176
  C:48DAH         LINE#         177
  C:48DAH         LINE#         178
  C:48E4H         LINE#         181
  C:48E9H         LINE#         182
  C:48E9H         LINE#         183
  C:48ECH         LINE#         184
  C:4901H         LINE#         185
  C:4916H         LINE#         186
  C:4926H         LINE#         187
  C:4936H         LINE#         188
  C:4946H         LINE#         189
  C:4956H         LINE#         190
  C:4956H         LINE#         193
  C:4965H         LINE#         194
  C:497AH         LINE#         195
  C:4986H         LINE#         196
  C:499BH         LINE#         197
  C:49A5H         LINE#         198
  C:49BAH         LINE#         199
  C:49CFH         LINE#         200
  C:49E4H         LINE#         201
  C:49F3H         LINE#         202
  C:49FFH         LINE#         203
  C:4A14H         LINE#         204
  C:4A34H         LINE#         205
  C:4A3EH         LINE#         206
  C:4A53H         LINE#         207
  C:4A68H         LINE#         208
  C:4A7DH         LINE#         209
  -------         ENDPROC       _SCREEN3
  -------         ENDMOD        SCREENS

  -------         MODULE        USER_ACTIONS
  C:0000H         SYMBOL        _ICE_DUMMY_
  B:00D8H.2       PUBLIC        CCF2
  B:00D8H.3       PUBLIC        CCF3
BL51 BANKED LINKER/LOCATER V4.02                                                      05/28/2008  17:48:13  PAGE 50


  B:00D8H.4       PUBLIC        CCF4
  C:5705H         PUBLIC        ActLEDblink
  B:00D0H.6       PUBLIC        AC
  B:00B0H.4       PUBLIC        T0
  B:00B0H.5       PUBLIC        T1
  B:00A8H.7       PUBLIC        EA
  B:00A8H.6       PUBLIC        EC
  B:00D8H.7       PUBLIC        CF
  B:0098H.7       PUBLIC        FE
  B:00E8H.1       PUBLIC        EADC
  B:0080H.0       PUBLIC        P0_0
  B:0090H.0       PUBLIC        P1_0
  B:0080H.1       PUBLIC        P0_1
  B:00A0H.0       PUBLIC        P2_0
  B:0090H.1       PUBLIC        P1_1
  B:0080H.2       PUBLIC        P0_2
  B:00B0H.0       PUBLIC        P3_0
  B:00A0H.1       PUBLIC        P2_1
  B:0090H.2       PUBLIC        P1_2
  B:0080H.3       PUBLIC        P0_3
  B:00C0H.0       PUBLIC        P4_0
  B:00B0H.1       PUBLIC        P3_1
  B:00A0H.2       PUBLIC        P2_2
  B:0090H.3       PUBLIC        P1_3
  B:0080H.4       PUBLIC        P0_4
  B:00D8H.6       PUBLIC        CR
  B:00C0H.1       PUBLIC        P4_1
  B:00B0H.2       PUBLIC        P3_2
  B:00A0H.3       PUBLIC        P2_3
  B:0090H.4       PUBLIC        P1_4
  B:0080H.5       PUBLIC        P0_5
  B:00C8H.6       PUBLIC        EXF2
  B:00B0H.7       PUBLIC        RD
  B:00B0H.3       PUBLIC        P3_3
  B:00A0H.4       PUBLIC        P2_4
  B:0090H.5       PUBLIC        P1_5
  B:0080H.6       PUBLIC        P0_6
  B:00B0H.4       PUBLIC        P3_4
  B:00A0H.5       PUBLIC        P2_5
  B:0090H.6       PUBLIC        P1_6
  B:0080H.7       PUBLIC        P0_7
  B:00E8H.0       PUBLIC        ECAN
  B:00A8H.4       PUBLIC        ES
  B:00B0H.5       PUBLIC        P3_5
  B:00A0H.6       PUBLIC        P2_6
  B:0090H.7       PUBLIC        P1_7
  B:00D0H.1       PUBLIC        UD
  B:00B0H.6       PUBLIC        P3_6
  B:00A0H.7       PUBLIC        P2_7
  B:00B0H.7       PUBLIC        P3_7
  B:0098H.0       PUBLIC        RI
  B:00D0H.7       PUBLIC        CY
  B:00B0H.2       PUBLIC        INT0
  B:0098H.1       PUBLIC        TI
  B:00B0H.3       PUBLIC        INT1
  C:0017H         PUBLIC        ActBackLEDoff
  B:00D0H.2       PUBLIC        OV
BL51 BANKED LINKER/LOCATER V4.02                                                      05/28/2008  17:48:13  PAGE 51


  B:00C8H.1       PUBLIC        C_T2
  B:00B0H.6       PUBLIC        WR
  B:00C8H.5       PUBLIC        RCLK
  B:00C8H.4       PUBLIC        TCLK
  B:00E8H.2       PUBLIC        ETIM
  B:00E8H.3       PUBLIC        ESPI
  B:0088H.1       PUBLIC        IE0
  B:0088H.3       PUBLIC        IE1
  C:001EH         PUBLIC        ActBackLEDon
  B:00C8H.0       PUBLIC        CP_RL2
  B:00A8H.1       PUBLIC        ET0
  B:00A8H.3       PUBLIC        ET1
  B:0088H.5       PUBLIC        TF0
  B:00A8H.5       PUBLIC        ET2
  B:0088H.7       PUBLIC        TF1
  B:0098H.2       PUBLIC        RB8
  B:00C8H.7       PUBLIC        TF2
  B:00A8H.0       PUBLIC        EX0
  B:0088H.0       PUBLIC        IT0
  B:00A8H.2       PUBLIC        EX1
  B:0098H.3       PUBLIC        TB8
  B:0088H.2       PUBLIC        IT1
  B:00D0H.0       PUBLIC        P
  B:0098H.7       PUBLIC        SM0
  B:0098H.6       PUBLIC        SM1
  B:0098H.5       PUBLIC        SM2
  B:00D0H.3       PUBLIC        RS0
  B:0088H.4       PUBLIC        TR0
  B:00D0H.4       PUBLIC        RS1
  B:0088H.6       PUBLIC        TR1
  B:00C8H.2       PUBLIC        TR2
  B:00C8H.3       PUBLIC        EXEN2
  B:0098H.4       PUBLIC        REN
  B:00B0H.0       PUBLIC        RXD
  B:00B0H.1       PUBLIC        TXD
  X:1740H         PUBLIC        ActLedBlinkN
  B:00D0H.5       PUBLIC        F0
  B:00D8H.0       PUBLIC        CCF0
  B:00D8H.1       PUBLIC        CCF1
  -------         PROC          ACTLEDBLINK
  -------         DO            ACTLEDBLINK
  X:172CH         SYMBOL        i
  -------         ENDDO         i
  C:5705H         LINE#         15
  C:5705H         LINE#         19
  C:5728H         LINE#         20
  C:5728H         LINE#         21
  C:5728H         LINE#         22
  C:572BH         LINE#         23
  C:572BH         LINE#         24
  C:572EH         LINE#         25
  C:573EH         LINE#         26
  -------         ENDPROC       ACTLEDBLINK
  -------         PROC          ACTBACKLEDOFF
  C:0017H         LINE#         31
  C:0017H         LINE#         32
  C:0017H         LINE#         33
BL51 BANKED LINKER/LOCATER V4.02                                                      05/28/2008  17:48:13  PAGE 52


  C:0019H         LINE#         34
  -------         ENDPROC       ACTBACKLEDOFF
  -------         PROC          ACTBACKLEDON
  C:001EH         LINE#         39
  C:001EH         LINE#         40
  C:001EH         LINE#         41
  C:0020H         LINE#         42
  -------         ENDPROC       ACTBACKLEDON
  -------         ENDMOD        USER_ACTIONS

  -------         MODULE        ?C?COPY
  C:3034H         PUBLIC        ?C?COPY
  -------         ENDMOD        ?C?COPY

  -------         MODULE        ?C?CLDPTR
  C:305AH         PUBLIC        ?C?CLDPTR
  -------         ENDMOD        ?C?CLDPTR

  -------         MODULE        ?C?CILDPTR
  C:3073H         PUBLIC        ?C?CILDPTR
  -------         ENDMOD        ?C?CILDPTR

  -------         MODULE        ?C?CSTPTR
  C:3095H         PUBLIC        ?C?CSTPTR
  -------         ENDMOD        ?C?CSTPTR

  -------         MODULE        ?C?IMUL
  C:30A7H         PUBLIC        ?C?IMUL
  -------         ENDMOD        ?C?IMUL

  -------         MODULE        ?C?SIDIV
  C:30B9H         PUBLIC        ?C?SIDIV
  -------         ENDMOD        ?C?SIDIV

  -------         MODULE        ?C?ILDIX
  C:30EFH         PUBLIC        ?C?ILDIX
  -------         ENDMOD        ?C?ILDIX

  -------         MODULE        ?C?ILDPTR
  C:3105H         PUBLIC        ?C?ILDPTR
  -------         ENDMOD        ?C?ILDPTR

  -------         MODULE        ?C?IILDPTR
  C:3130H         PUBLIC        ?C?IILDPTR
  -------         ENDMOD        ?C?IILDPTR

  -------         MODULE        ?C?ISTPTR
  C:3168H         PUBLIC        ?C?ISTPTR
  -------         ENDMOD        ?C?ISTPTR

  -------         MODULE        ?C?ISTOPTR
  C:3187H         PUBLIC        ?C?ISTOPTR
  -------         ENDMOD        ?C?ISTOPTR

  -------         MODULE        ?C?LMUL
  C:31B4H         PUBLIC        ?C?LMUL
  -------         ENDMOD        ?C?LMUL
BL51 BANKED LINKER/LOCATER V4.02                                                      05/28/2008  17:48:13  PAGE 53



  -------         MODULE        ?C?SLDIV
  C:5749H         PUBLIC        ?C?SLDIV
  -------         ENDMOD        ?C?SLDIV

  -------         MODULE        ?C?SLSHR
  C:3203H         PUBLIC        ?C?SLSHR
  -------         ENDMOD        ?C?SLSHR

  -------         MODULE        ?C?OFFXADD
  C:3217H         PUBLIC        ?C?OFFXADD
  -------         ENDMOD        ?C?OFFXADD

  -------         MODULE        ?C?PSTOPTR
  C:3223H         PUBLIC        ?C?PSTOPTR
  -------         ENDMOD        ?C?PSTOPTR

  -------         MODULE        ?C?ICALL
  C:327CH         PUBLIC        ?C?ICALL
  -------         ENDMOD        ?C?ICALL

  -------         MODULE        PRINTF
  D:0022H         PUBLIC        ?_PRINTF517?BYTE
  D:0022H         PUBLIC        ?_PRINTF?BYTE
  D:0022H         PUBLIC        ?_SPRINTF517?BYTE
  D:0022H         PUBLIC        ?_SPRINTF?BYTE
  C:3D3EH         PUBLIC        _PRINTF
  C:3D3EH         PUBLIC        _PRINTF517
  C:3D38H         PUBLIC        _SPRINTF
  C:3D38H         PUBLIC        _SPRINTF517
  -------         ENDMOD        PRINTF

  -------         MODULE        RAND
  D:003EH         PUBLIC        ?SRAND?BYTE
  C:578DH         PUBLIC        RAND
  C:57C4H         PUBLIC        _SRAND
  -------         ENDMOD        RAND

  -------         MODULE        ?C?STRCPY
  C:334EH         PUBLIC        ?C?STRCPY
  -------         ENDMOD        ?C?STRCPY

  -------         MODULE        ?C?MEMSET
  C:336BH         PUBLIC        ?C?MEMSET
  -------         ENDMOD        ?C?MEMSET

  -------         MODULE        ?C?CLDOPTR
  C:3397H         PUBLIC        ?C?CLDOPTR
  -------         ENDMOD        ?C?CLDOPTR

  -------         MODULE        ?C?UIDIV
  C:33C4H         PUBLIC        ?C?UIDIV
  -------         ENDMOD        ?C?UIDIV

  -------         MODULE        ?C?IILDX
  C:3419H         PUBLIC        ?C?IILDX
  -------         ENDMOD        ?C?IILDX
BL51 BANKED LINKER/LOCATER V4.02                                                      05/28/2008  17:48:13  PAGE 54



  -------         MODULE        ?C?ULDIV
  C:346BH         PUBLIC        ?C?ULDIV
  -------         ENDMOD        ?C?ULDIV

  -------         MODULE        ?C?PLDIIDATA
  C:34FDH         PUBLIC        ?C?PLDIIDATA
  -------         ENDMOD        ?C?PLDIIDATA

  -------         MODULE        ?C?PSTIDATA
  C:350DH         PUBLIC        ?C?PSTIDATA
  -------         ENDMOD        ?C?PSTIDATA

  -------         MODULE        ?C?PSTXDATA
  C:3516H         PUBLIC        ?C?PSTXDATA
  -------         ENDMOD        ?C?PSTXDATA

  -------         MODULE        ?C?PSTPDATA
  C:351FH         PUBLIC        ?C?PSTPDATA
  -------         ENDMOD        ?C?PSTPDATA

  -------         MODULE        ?C?CCASE
  C:3528H         PUBLIC        ?C?CCASE
  -------         ENDMOD        ?C?CCASE

  -------         MODULE        PUTCHAR
  C:58DCH         PUBLIC        _PUTCHAR
  -------         ENDMOD        PUTCHAR

*** WARNING L15: MULTIPLE CALL TO SEGMENT
    SEGMENT: ?PR?_ADDACTION?BUTTONS
    CALLER1: ?PR?INTTIMER0?BUTTONS
    CALLER2: ?C_C51STARTUP

*** WARNING L15: MULTIPLE CALL TO SEGMENT
    SEGMENT: ?PR?_E3D_MAKE_MOVE_ROTATE_TRANSFORM?E3D_DEMO
    CALLER1: ?PR?INTTIMER0?BUTTONS
    CALLER2: ?C_C51STARTUP

*** WARNING L15: MULTIPLE CALL TO SEGMENT
    SEGMENT: ?PR?_E3D_DRAWOBJECT?E3D_DEMO
    CALLER1: ?PR?INTTIMER0?BUTTONS
    CALLER2: ?C_C51STARTUP

*** WARNING L15: MULTIPLE CALL TO SEGMENT
    SEGMENT: ?PR?_E3D_ROTATE?E3D_DEMO
    CALLER1: ?PR?INTTIMER0?BUTTONS
    CALLER2: ?C_C51STARTUP

*** WARNING L15: MULTIPLE CALL TO SEGMENT
    SEGMENT: ?PR?_E3D_RANDOMMOVE?E3D_DEMO
    CALLER1: ?PR?INTTIMER0?BUTTONS
    CALLER2: ?C_C51STARTUP

LINK/LOCATE RUN COMPLETE.  5 WARNING(S),  0 ERROR(S)
